:020000040800F2
:10000000B8800020210300080539000811300008DD
:100010009D3700086907000815430008000000002C
:100020000000000000000000000000002D02000899
:10003000730D00080000000089020008A73A0008BC
:100040003B0300083B0300083B0300083B03000898
:100050003B0300083B0300083B0300083B03000888
:100060003B030008750D00087B0D00083B030008EA
:10007000C90B00083B0300083B0300083B030008D2
:10008000D50B0008E10B00083B0300083B03000808
:100090006D070008790700083B030008810D000880
:1000A0003B0300083B0300083B0300083B03000838
:1000B0003B0300083B0300083B0300083B03000828
:1000C0003B0300083B0300083B0300083B03000818
:1000D0003B030008D54200083B030008ED4200083E
:1000E0003B0300083B0300083B0300083B030008F8
:1000F0003B0300083B0300083B0300083B030008E8
:100100003B0300083B0300083B0300083B030008D7
:100110003B0300083B0300083B030008653B000865
:100120003B030008ED0B0008F90B0008050C000864
:100130003B0300083B0300083B0300083B030008A7
:1001400085070008910700083B0300083B030008EF
:10015000110C00081D0C0008290C000809430008B8
:100160003B0300083B0300083B0300083B03000877
:100170003B0300083B0300083B03000800000000AD
:100180003B0300083B03000800F002F800F03EF8D3
:100190000AA090E8000C82448344AAF10107DA45E2
:1001A00001D100F033F8AFF2090EBAE80F0013F0F6
:1001B000010F18BFFB1A43F0010318473C6D000004
:1001C0005C6D0000103A24BF78C878C1FAD8520795
:1001D00024BF30C830C144BF04680C6070470000C1
:1001E0000023002400250026103A28BF78C1FBD840
:1001F000520728BF30C148BF0B6070471FB506F0DB
:1002000006FE00F03AF91FBD10B510BD00F01CFA53
:100210001146FFF7F3FF04F039FB00F03AFA03B49C
:10022000FFF7F2FF03BC00F03DFA00002C4B196809
:100230000868B0E8F04F80F30988BFF36F8F4FF084
:10024000000080F311887047000000000848006833
:10025000006880F308884FF0000080F3148862B6CD
:1002600061B6BFF34F8FBFF36F8F00DF00BF00BFDA
:1002700008ED00E0DFF80C00016841F47001016056
:10028000704700BF88ED00E0EFF30980BFF36F8F88
:10029000134B1A681EF0100F08BF20ED108A20E9DA
:1002A000F04F106009B44FF0500080F31188BFF395
:1002B0004F8FBFF36F8F05F087FB4FF0000080F387
:1002C000118809BC19680868B0E8F04F1EF0100FDB
:1002D00008BFB0EC108A80F30988BFF36F8F7047B6
:1002E00018000020EFF30580704700000B49D1F89B
:1002F00000C04A685CF8043B1068184442F8040BDC
:100300008C4528BFA1F1DC0C8A4228BFA1F1DC0298
:10031000C1F800C04A6020F0004070474C7A0020CD
:100320000948804709480047FEE7FEE7FEE7FEE789
:10033000FEE7FEE7FEE7FEE7FEE7FEE704480549C5
:10034000054A064B70470000553B0008890100082C
:10035000B87A0020B8800020B87C0020B87C00204B
:1003600053EA020C00F069802DE9F04B4FF00006D3
:10037000002B1FBFB3FA83F503FA05F424FA05F640
:100380005E4012BF1643B2FA82F502FA05F4C5F1D7
:1003900020051EBF22FA05FC44EA0C04203556EA6B
:1003A000044C4FEA144418BF641C4FF000084FF08F
:1003B0000009904271EB030C39D3002919BFB1FA3F
:1003C00081F701FA07F6B0FA80F700FA07F6C7F1ED
:1003D00020071EBF20FA07FC46EA0C062037B6FBB2
:1003E000F4FCA7EB0507103F07F01F0BCBF120062D
:1003F0000CFA0BFB2CFA06F644BFB3460026202F5E
:10040000A4BF5E464FF0000B5BEA060C08BF4FF03E
:10041000010B19EB0B09ABFB027C48EB0608C01B78
:1004200006FB02CC0BFB03CC71EB0C01C1E70B46C6
:10043000024641464846BDE8F08B13B54FF0000038
:100440004FF00001AFF30080BDE81C407047000092
:100450000B4910B5A1F17C020A4CC2E937123721D1
:1004600006E000EB104342F82130074B00FB03404D
:100470000B1EA1F10101F4DC10BD0120E8E7000032
:10048000EC790020E119D666CD0D0100032A40F277
:10049000308010F0030C00F0158011F8013BBCF126
:1004A000020F624498BF11F801CB00F8013B38BF3E
:1004B00011F8013BA2F1040298BF00F801CB38BF4C
:1004C00000F8013B11F0030300F06280083AC0F02D
:1004D000088051F8043B083A51F804CBA0E8081012
:1004E000F5E7121D5CBF51F8043B40F8043BAFF345
:1004F0000080D20724BF11F8013B11F801CB48BF9F
:1005000011F8012B24BF00F8013B00F801CB48BFD4
:1005100000F8012B704702F0FF0343EA032242EA8E
:10052000024200F069B84FF0000200B5134694464D
:100530009646203922BFA0E80C50A0E80C50B1F13B
:100540002001BFF4F7AF090728BFA0E80C5048BF4F
:100550000CC05DF804EB890028BF40F8042B08BFED
:10056000704748BF20F8022B11F0804F18BF00F8E9
:10057000012B704770477047704710B500F05CF86A
:10058000006810BD10B5044600F056F8046010BDB8
:1005900010B5203AC0F00B80B1E81850203AA0E81E
:1005A0001850B1E81850A0E81850BFF4F5AF5FEA52
:1005B000027C24BFB1E81850A0E8185044BF18C905
:1005C00018C0BDE810405FEA827C24BF51F8043BAC
:1005D00040F8043B08BF7047D20728BF31F8023B00
:1005E00048BF11F8012B28BF20F8023B48BF00F894
:1005F000012B70474FF000020429C0F0128010F068
:10060000030C3FF492AFCCF1040CBCF1020F18BF05
:1006100000F8012BA8BF20F8022BA1EB0C01FFF77B
:1006200084BF5FEAC17C24BF00F8012B00F8012BD6
:1006300048BF00F8012B704700487047547A0020EB
:1006400000487047547A00207546FFF7F9FFAE4620
:1006500005006946534620F00700854618B020B5CE
:10066000FFF76CFEBDE820404FF000064FF000079A
:100670004FF000084FF0000B21F00701AC46ACE84A
:10068000C009ACE8C009ACE8C009ACE8C0098D46B7
:10069000704710B50446AFF300802046BDE8104017
:1006A000FFF7BDBD01491820ABBEFEE726000200E2
:1006B0007047B1EE601AB4EEC10AF1EE10FA02D240
:1006C000B0EE410A7047B4EEE00AF1EE10FAF9DD3F
:1006D000B0EE600A7047000018B1012803D0002076
:1006E000704702487047024870470000100400201D
:1006F000A004002038B5016804460868C00619D572
:10070000086848680090204603F09AFC0A4D00EB08
:10071000C00005EB8000006A00280BD0204603F0E3
:100720008FFC00EBC00005EB8000006A01B0BDE863
:100730003040004738BD00001C75002032B102284F
:1007400001D2092905D34FF0FF3070476FF0010047
:100750007047044B00EBC00003EB800040F8212001
:10076000002070471C750020FEE70000014800F0E3
:1007700023BB0000C4000020014800F01DBB0000A6
:10078000C4000020014800F017BB0000EC0000206E
:10079000014800F011BB0000EC00002050B10068DF
:1007A0000549884201D1002070470449884201D19F
:1007B000012070470320704700640040006800403B
:1007C00070B504002DED048B16460D466FF0010048
:1007D0007DD0002D7BD02068301A00EE100AB8EED4
:1007E000400ADFED880A3246204680EE201A84ED6A
:1007F000011A2660297800F035F9207CDFED828A25
:10080000072838D2DFE800F010041010100910009B
:10081000C4ED098AC4ED0A8A2DE095ED010A84ED44
:10082000090A95ED020A24E0E06894ED0C0AD0ED87
:10083000000A30EE609AB0EE490A03F097FDF0EE40
:10084000400AB0EE490AB0EE608A03F05BFED5EDD7
:10085000010A95ED021A60EE880A40EE410AC4EDE5
:10086000090AD5ED010A20EE800AD5ED020A08EE4C
:10087000200A84ED0A0A217C04F14800072921D2CC
:10088000DFE801F00404070F2F040700C4ED0B8A12
:1008900018E0E168D4ED011AD4ED0C0A91ED000ADC
:1008A0000AE0E168D4ED011AD4ED0C0A91ED000ADA
:1008B0009FED561A30EE010AB0EE681A03F024F8E4
:1008C00084ED0B0A94F911309FED510A00E095E098
:1008D00004F1240104F11200226C02F061FF0025F2
:1008E00087E09FED4C9A9FED4C8A00EE106AB8EEBF
:1008F000400A10EE100A06F0E3F99FED481B53EC96
:10090000112B06F0DFF805F013FF00EE100A03F0DC
:10091000F9FDDFED440A20EE200AB0EEC00A30EE09
:10092000090AB4EEC80AF1EE10FA01DDB0EE480A89
:10093000D4ED0F0A20EE200AC2E7606B00EB8500C1
:1009400090ED000AD4F8840000EB451002F062FB41
:10095000606BF0EE400A00EB850080ED000A207C21
:10096000072832D2DFE800F02B04040404041B0043
:10097000206CC5EB051100EB8500D4ED011A90ED5C
:10098000000A606CB0EE681A00EB810002F0BCFF58
:10099000D4F88C0000EB850080ED000A15E0206C97
:1009A000DFED210A00EB850090ED000AD4F88C0001
:1009B00080EE201A00EB850080ED001A05E0D4F8E7
:1009C0008C0000EB8500C0ED008AD4F88C0000EBB1
:1009D000850090ED000A54F8880F00EB451002F0F6
:1009E00019FB606800EB85006D1C80ED000AEDB21C
:1009F000883C94F91100A8429FDC0020BDEC048BD8
:100A000070BD000000007A4400000000AB611C3F94
:100A100000C0DA459A99193FCDCC4C3FFCA9F1D2E0
:100A20004D62503FCDCC4C3E00A00C4670B50E46FA
:100A3000050016D0002E14D000240EE0D5F88C103E
:100A400004EB840001EB840106EB001091ED000A39
:100A5000083002F06FFB641CE4B295F91100A0426B
:100A6000ECDC70BD70B50E462DED028B040006D097
:100A7000207CB04206D10020BDEC028B70BD6FF02F
:100A80000100F9E7042E11D104280FD01046FFF71A
:100A9000DFFCFFF72BFCC00701D0701F00E0012036
:100AA00000EE100AB8EEC00A84ED0F0A00259FED93
:100AB000118A18E0606CC5EB051100EB810002F0B3
:100AC000D5FFD4F88400B0EE480A00EB451002F0E0
:100AD000CFFAD4F88800B0EE480A00EB451002F0D7
:100AE000C7FA6D1CEDB294F91100A842E2DC26743D
:100AF000C1E700000000000070B504000D466FF073
:100B000001003DD0002D3BD0A06890F84C1005F5B9
:100B1000B07031B102F0D0FADFED1A0A30EEC00A3F
:100B200001E002F0C9FA84ED0C0A00209FED160ADC
:100B300021E000BF00EB800105EB011108310ED070
:100B4000626BD1ED030A02EB8002C2ED000AD1ED27
:100B5000040AA16B01EB8001C1ED000A09E0616BA1
:100B600001EB800181ED000AA16B01EB800181EDB9
:100B7000000A401CC0B294F911108142DADC002056
:100B800070BD0000DB0FC9400000000030EE600ABD
:100B9000B5EEC01AF1EE10FA0ADDF6EE000A61EECB
:100BA000200AB4EEE00AF1EE10FA02DD30EE410A5E
:100BB0007047F1EE600AB4EEE00AF1EE10FAF7D2F7
:100BC00030EE010A70470000014800F071BC0000DF
:100BD000B0060020014800F06BBC0000F0050020CA
:100BE000014800F065BC000050060020014800F0FC
:100BF0005FBC000010070020014800F059BC000055
:100C0000C0020020014800F053BC00002003002077
:100C1000014800F04DBC000030050020014800F004
:100C200047BC000070070020014800F041BC0000F4
:100C30009005002001681823CAB2103AB2FBF3F203
:100C4000054B6FF30901032A9B5CC36500D9091D9D
:100C50008165084670470000486E000810B50146DF
:100C600000208B698A6A4FF0C07453B1B3F5005FFE
:100C700015D072B1012A0CD0022A0AD0032A09D158
:100C800004E01AB1012A06D0022A03D1C96AC901B7
:100C900000D5012010BDC96AA142FAD010BD002ABA
:100CA000F7D0012AF2D0022AF3D0032AF3D010BDE4
:100CB00030B50468256825F48025256004686360E4
:100CC0008368402B036803D099600068C26030BD20
:100CD0009A600068C16030BD70B56FF0010590B1D9
:100CE0000A4C207810B16FF0020070BD03F041FF94
:100CF000606040B1064A03210120FFF71FFD01207B
:100D00002070002070BD284670BD0000A0000020AB
:100D1000310D000810B538B1002100F8241B342132
:100D2000FFF701FC002010BD6FF0010010BD0000B6
:100D300002480121406803F097BE0000A000002097
:100D400010B504460120FFF7C7FC132204F110017F
:100D500002F014F9002801D04FF0FF3010BD10B59B
:100D600002460121084603F0B9FE012800D0002008
:100D700010BD7047082000F00DBD102000F00ABD26
:100D8000202000F007BD72B6FEE7000010B5FFF7A7
:100D900005FD03280CD000EB800101EBC0010548E4
:100DA00000EB8100006B002802D0BDE81040004736
:100DB00010BD0000B47400202DE9F05F0546006806
:100DC00000244669D0F804908768D0F80CB0D0F8B9
:100DD00010A0D0F81880F10748D0F90714D00121ED
:100DE0008160B80703D5284600F084FA0CE0780744
:100DF00002D54FF4006407E0380702D54FF4805461
:100E000002E0284600F060FAF80516D529684FF48C
:100E100080708860B80503D5284600F095FA0CE08C
:100E2000780502D544F4005407E0380502D544F4AF
:100E3000804402E0284600F071FAF80316D52968CC
:100E40004FF480308860B80303D5284600F0A8FA34
:100E50000CE0780302D544F4004407E0380302D5DF
:100E600044F4803402E0284600F084FA300707D5C5
:100E70005FEACB6004D52968102044F40074C86090
:100E800070074FF0080707D55FEA0B7004D5286894
:100E9000C760284600F0AAF9B00706D52868C068E0
:100EA000800702D0284600F0B7F9700607D55FEA40
:100EB000CA6004D52968102044F480640861B00633
:100EC00007D55FEA0A7004D528680761284600F054
:100ED000B9F9F00606D528680069800702D02846CF
:100EE00000F0C6F9B00308D55FEAC96005D52968E6
:100EF00010204860284600F0D1F9F00307D55FEADA
:100F0000097004D528684760284600F05FFA30046D
:100F100046D55FEA497040D5F00504D55FEAC87050
:100F200001D044F00104B00504D55FEA887001D512
:100F300044F00204700504D55FEA487001D544F01E
:100F40000404300529D518F0700F26D008F0700081
:100F5000402815D006DC102809D020280AD03028D7
:100F600016D10AE050280ED0602811D10EE044F0CE
:100F700008040DE044F010040AE044F0200407E007
:100F800044F0400404E044F0800401E044F4807440
:100F90002868816921F07001816129680420486016
:100FA000002C05D0686A204368622846FFF7EEFEF1
:100FB000BDE8F09F70B5040003D094F8200010B194
:100FC00004E0012070BD204600F082F8206801682E
:100FD00041F00101016000F0E7FC0546052604E050
:100FE00000F0E2FC401B0A2811D820684068C007C6
:100FF000F6D02068016821F00201016000F0D4FC05
:1010000005460BE000F0D0FC401B0A2806D9606AB8
:1010100040F40030606284F82060D2E720684068C5
:101020008007EFD4207E0128206801683DD021F0A0
:1010300080010160607E01282068016838D021F0BD
:1010400040010160A07E01282068016833D021F0B2
:1010500020010160E07E0128206801682ED041F067
:1010600010010160207F01282068016829D021F04B
:1010700008010160607F01282068016824D021F008
:1010800004010160D4E902010843D4E904121143C8
:1010900008436168491E08432168C86100206062F6
:1010A000012084F82000002070BD41F08001C0E7DD
:1010B00041F04001C5E741F02001CAE721F01001ED
:1010C000CFE741F00801D4E741F00401D9E700007F
:1010D000F0B587B0044614216846FFF724FA3E4B6A
:1010E0003E48DFF8F0E01968D4F800C03B4A032519
:1010F0000226092710300024491CF4452AD1196022
:10110000012907D1016841F000710160006800F019
:1011100000700590106840F0080010601068CDE97C
:10112000005600F00800CDE9047069462C48CDE96E
:10113000024500F03BFB00220821142000F0F6FDE0
:10114000142000F0E5FD00220521152000F0EEFD41
:1011500015203AE0DFF88CE0F44538D1D0F800C033
:101160004CF0806CC0F800C0D0F800C001290CF031
:10117000806CCDF814C0196007D1016841F000718E
:101180000160006800F000700590106840F00200F7
:101190001060106802AB00F0020005906020CDE9FD
:1011A000000683E8B00069460F4800F0FFFA00220D
:1011B0000521402000F0BAFD402000F0A9FD0022EA
:1011C0000521412000F0B2FD412000F0A1FD07B053
:1011D000F0BD0000006400400400002030380240F0
:1011E000000C0240006800400004024010B5FFF708
:1011F000D5FA03280CD000EB800101EBC0010548B3
:1012000000EB8100C069002802D0BDE81040004713
:1012100010BD0000B474002010B5FFF7BFFA03281A
:101220000CD000EB800101EBC001054800EB810010
:101230008069002802D0BDE81040004710BD0000C2
:10124000B474002010B5FFF7A9FA03280CD000EB06
:10125000800101EBC001054800EB8100406A0028D5
:1012600002D0BDE81040004710BD0000B47400205B
:1012700010B5FFF793FA03280CD000EB800101EBC7
:10128000C001054800EB8100006A002802D0BDE8DB
:101290001040004710BD0000B474002010B5FFF7E7
:1012A0007DFA03280CD000EB800101EBC00105485A
:1012B00000EB8100806A002802D0BDE810400047A2
:1012C00010BD0000B474002010B5FFF767FA0328C2
:1012D0000CD000EB800101EBC001054800EB810060
:1012E000C068002802D0BDE81040004710BD0000D3
:1012F000B474002010B5FFF751FA03280BD000EBAF
:10130000800101EBC001044850F82100002802D000
:10131000BDE81040004710BDB474002010B5FFF7C1
:101320003DFA03280CD000EB800101EBC001054819
:1013300000EB81000069002802D0BDE810400047A2
:1013400010BD0000B474002010B5FFF727FA032881
:101350000CD000EB800101EBC001054800EB8100DF
:101360004068002802D0BDE81040004710BD0000D2
:10137000B474002010B5FFF711FA03280CD000EB6D
:10138000800101EBC001054800EB810040690028A5
:1013900002D0BDE81040004710BD0000B47400202A
:1013A00010B5FFF7FBF903280CD000EB800101EB2F
:1013B000C001054800EB81008068002802D0BDE82C
:1013C0001040004710BD0000B474002010B5FFF7B6
:1013D000E5F903280CD000EB800101EBC0010548C2
:1013E00000EB8100C06A002802D0BDE81040004731
:1013F00010BD0000B47400202DE9F0410446876D53
:1014000000F0D2FA064694F835000025022806D0EE
:101410008020606584F834500120BDE8F0812068A8
:10142000016821F0160101602068416921F0800106
:101430004161206C08B9A06C20B12068016821F0DE
:10144000080101602068016821F0010101600CE0E1
:1014500000F0AAFA801B052807D920206065032028
:1014600084F8350084F83450D7E720680068C00756
:10147000EED194F85C103F208840B860012084F8D9
:10148000350084F834500020C7E790F83510022961
:1014900003D08021416501207047052180F8351077
:1014A0000068016821F00101016000207047000020
:1014B0002DE9F84304464FF00009CDF80090634849
:1014C0004FF41651A56D0068B0FBF1F72E6894F843
:1014D0005C10082000FA01F131420FD021680A683F
:1014E00052070BD50A6822F004020A6094F85C10D7
:1014F0008840A860606D40F00100606594F85C1061
:101500004FF0010808FA01F0304208D0216849691B
:10151000090604D5A860606D40F00200606594F88B
:101520005C1004208840304208D02168096889078F
:1015300004D5A860606D40F00400606594F85C100C
:1015400010208840304218D021680968090714D556
:10155000A86020680168490304D50068000308D525
:10156000A16C07E00168C90503D4016821F00801F6
:101570000160216C09B12046884794F85C10202056
:101580008840304231D021680968C9062DD5A8604D
:1015900094F8350005282068016806D0490347D52E
:1015A000006800031DD4616C1CE021F0160101608D
:1015B0002068416921F080014161206C08B9A06C6C
:1015C00020B12068016821F00801016094F85C10E6
:1015D0003F208840A86084F8358084F83490216DDD
:1015E0001FE0E16B09B120468847606D00282BD0D1
:1015F000606DC00714D0052084F8350020680168AC
:1016000021F0010101600098401C0090B84203D80D
:1016100020680068C007F6D184F8358084F83490DB
:10162000E16C002910D001B02046BDE8F043084726
:101630000168C905D5D4016821F01001016084F862
:10164000358084F83490CCE7BDE8F883140000209E
:101650002DE9F041044600F0A7F906465CB10220EE
:1016600084F83500002584F834502068016821F0A2
:10167000010101600DE00120BDE8F08100F094F966
:10168000801B052805D920206065032084F83500DB
:10169000F2E720680068C007F0D12268116820488E
:1016A0000140D4E901031843D4E903363343184316
:1016B00063691843A3691843E3691843236A18430D
:1016C0000843616A042903D1D4E90B131943084381
:1016D000106020684069666A20F0070130460E43BA
:1016E000012704280CD1A06A0643E06A40B12046D5
:1016F000FFF7B4FA20B14020606584F83570BAE78E
:10170000206846612046FFF795FA94F85C203F2157
:1017100091408160656584F835700020ACE7000079
:101720003F8010F02DE9F0410446866D90F83400BA
:10173000002501280DD0012084F8340094F835707C
:101740000020012F07D084F8340002252846BDE888
:10175000F0810220FBE7022784F83570606520469F
:10176000FFF7A6FA94F85C103F208840B06020682C
:10177000016841F016010160206C20B12068016809
:1017800041F0080101602068016841F00101016039
:10179000DCE77047044910B50A68024202D00860CD
:1017A000FFF7F7FF10BD0000143C01402DE9F84F92
:1017B000DFF8BCA10022012503264FF00F090AF132
:1017C000040BAAF1040E00BF0B6805FA02F42340D3
:1017D000A34270D10F7907F00307012F01D0022F28
:1017E00016D187684FEA420806FA08FC27EA0C0778
:1017F000D1F80CC00CFA08FC4CEA070CC0F808C081
:101800004768A7430C79C4F3001494403C434460F8
:101810000C79E443A4070AD0C4684FEA420C06FAE4
:101820000CF7BC438F6807FA0CF72743C7600C79A5
:1018300004F00304022C12D1D40800EB840CDCF871
:1018400020405707FF0E09FA07F824EA0804D1F8E8
:10185000108008FA07F848EA0408CCF820800468E9
:101860004FEA420C06FA0CF7BC430F7907F0030766
:1018700007FA0CF7274307604C6814F4403F70D018
:101880003C4C276847F480472760246822F0030710
:1018900004F480440094384C07EB040CDCF808484E
:1018A00097074FEA177809FA08F7BC43334FB84255
:1018B00002D1002724E054E0314FB84201D1012782
:1018C0001EE0304FB84201D1022719E02E4FB84236
:1018D00001D1032714E02D4FB84201D104270FE0B6
:1018E0002B4FB84201D105270AE02A4FB84201D157
:1018F000062705E0284FB84201D1072700E0082756
:1019000007FA08F72743CCF80878DAF8004057467A
:10191000D1F804C09C435FEACC2C00D51C433C604A
:10192000DBF800405F46D1F804C09C435FEA8C2C92
:1019300000D51C433C60DEF800407746D1F804C077
:101940009C435FEA8C3C00D51C433C60084F083F39
:101950003C68D1F804C09C435FEACC3C00D51C43F2
:101960003C60521C102AFFF42FAFBDE8F88F000036
:10197000083C014044380240003001400000024071
:101980000004024000080240000C02400010024027
:101990000014024000180240001C02400AB181619C
:1019A00070470904FBE700000148806870470000A9
:1019B0000800002070B5040025D094F83D000025F3
:1019C00020B984F83C50204600F0B8F8242084F870
:1019D0003D002068016821F0010101602068016874
:1019E00041F4004101602068016821F40041016078
:1019F00000F068FA4D4A6168914201D84C4900E014
:101A00004C49884201D2012070BD4B492368B0FB8C
:101A1000F1F15E6826F03F060E435E606368934214
:101A200006D94FF4967359434FF47A73B1FBF3F12F
:101A30002368491C1E6A26F03F063143196261681B
:101A4000914210D84900401EB0FBF1F2521CC2F383
:101A50000B02042A01D2042022E0B0FBF1F0401C6A
:101A6000C0F30B001CE0A268F2B301EBC10303EB6F
:101A70000116431EB3FBF6F35B1C43F480431B05C6
:101A800049D092B301EBC10202EB0111401EB0FB41
:101A9000F1F0401CC0F30B0040F4804040F40040E3
:101AA0002168CA694CF6FF739A431043C861D4E9B0
:101AB000071001432068026822F0C0021143016050
:101AC000D4E9030101432068826848F2FF339A4356
:101AD00011438160D4E9050108432168CA6822F0F6
:101AE000FF021043C86001E00EE016E020680168C4
:101AF00041F0010101602564202084F83D00256348
:101B000084F83E50002070BD01EB4106431EB3FB3C
:101B1000F6F35B1CB3E70120C2E701EB4101401E75
:101B2000B0FBF1F0401CC0F30B00B7E7A08601004A
:101B300080841E0000093D0040420F002DE9F04165
:101B400086B0044614216846FEF7EDFC22683A4C44
:101B5000384B0021384812260325042710349A42B6
:101B600019D1026842F002020260006802AA00F085
:101B70000200059082E8A2002802CDE9000669462D
:101B80002E48FFF713FE206840F400102060206804
:101B900000F400101AE02A4B9A421BD1026842F06E
:101BA00020020260006802AA00F020000590CDE942
:101BB000005682E8A20069462248FFF7F7FD206838
:101BC00040F480002060206800F48000059006B09A
:101BD000BDE8F0811C4B9A42F9D18846016841F07A
:101BE00004010160016801F004010591016841F000
:101BF000010101600068694600F001000590501580
:101C00008DE84101CDE903571048FFF7CFFD4FF4B0
:101C100080708DE84101CDE9035769460C48FFF714
:101C2000C5FD206840F400002060206800F400003A
:101C3000CCE700000054004030380240000402406D
:101C40000058004000140240005C004000080240C0
:101C500000000240024881680278114481607047A8
:101C6000080000200B4810B5016841F400710160C4
:101C7000016841F480610160016841F48071016094
:101C8000032000F073F80F2000F006F800F024F8AD
:101C9000002010BD003C024070B50D4D04464FF4CD
:101CA0007A712878B1FBF0F00A490968B1FBF0F0CD
:101CB00000F016FC48B9102C07D200222146501E15
:101CC00000F034F800206C6070BD012070BD000091
:101CD00008000020140000200C4882B0016841F484
:101CE00080410160006800F4804000900748001FB8
:101CF000016841F0805101600068002200F08050CE
:101D000000900F21901E02B000F010B8443802403D
:101D1000002809DB00F01F020121914040098000EA
:101D200000F1E020C0F8001170470000F0B40E4B45
:101D30001B680C46C3F30223C3F10705042D00D929
:101D40000425191D072901D2002300E0DB1E01260E
:101D500006FA05F1491E214099409E40761E164024
:101D60003143F0BC02F0F1BA0CED00E0064900F09E
:101D7000070208684FF6FF03184040EA0220034AB2
:101D800010430860704700000CED00E00000FA0509
:101D90002DE9F0470E46050065D0DFF81481D8F82C
:101DA0000000F7B200F00700B04207D288F80070D8
:101DB000D8F8000000F00700B04254D128683D4C2C
:101DC000810712D5400703D5206840F4E050206019
:101DD0002878000703D5206840F460402060206820
:101DE000A96820F0F000084320602878C0072DD0B3
:101DF000304968680839012812D0022813D0032816
:101E000011D00968890700292DDA216821F0030122
:101E100001432160FFF7C8FD814641F2883A0EE098
:101E200009688903EFE709688901ECE7FFF7BCFD62
:101E3000A0EB0901514502D90320BDE8F0872068D5
:101E4000696800F00C00B0EB810FEFD1D8F80010FA
:101E5000404601F00701B14207D90770006800F061
:101E60000700B04201D00120E7E72878400705D5F8
:101E70002068E96820F4E0500843206028780007D3
:101E800006D52068296920F4604040EAC10020603E
:101E900000F038F82168084AC1F30311515CC840CA
:101EA0000649086006480068FFF7F6FE0020C4E710
:101EB000003C024008380240506E00081400002028
:101EC0000C0000200448054900680968044AC1F371
:101ED0008221515CC840704714000020083802403D
:101EE000606E00080448054900680968044AC1F3A7
:101EF0004231515CC840704714000020083802404D
:101F0000606E0008154810B5006810F00C02144807
:101F100013D01449042A0FD0082A0ED10F4C241FC5
:101F20002268236802F03F025B0207D52068C0F3F5
:101F30008810A0FB010106E0084610BD2168C1F32E
:101F40008811A1FB00010023FEF70AFA2168C1F302
:101F50000141491C4900B0FBF1F010BD08380240B6
:101F60000024F400001BB7002DE9F84F04006ED0E8
:101F70002078DFF84C93C007A9F104054AD009F195
:101F800004000168C1F38101012908D00068C0F391
:101F9000810002280AD1D9F80000400206D528683D
:101FA000800337D560680028E1D033E06068B0F581
:101FB000803F10D0B0F5A02F286810D020F48030DA
:101FC0002860286820F4802028606068A8B1FFF7A6
:101FD000EBFC06460DE0286840F48030F4E740F45E
:101FE00080202860F7E700BFFFF7DEFC801B642835
:101FF00073D828688003F7D50CE0FFF7D5FC0646B8
:1020000005E000BFFFF7D0FC801B6428F0D82868EB
:102010008003F7D42078DFF8AC8280074FF0000A05
:102020003ED5A748001D016811F00C0F08D00068CC
:10203000C0F3810002280BD1D9F80000400207D478
:102040002868800716D5E068012800D112E033E146
:10205000E068B8B10120C8F80000FFF7A5FC06460B
:1020600005E000BFFFF7A0FC801B0228C0D828684D
:102070008007F7D52868216920F0F80040EAC10000
:1020800028600DE0C8F800A0FFF78EFC064604E0CB
:10209000FFF78AFC801B02281FD828688007F7D426
:1020A0002078000722D5864F87486169703771B163
:1020B00001210160FFF778FC064604E0FFF774FC9D
:1020C000801B022809D838688007F7D50EE0C0F8D1
:1020D00000A0FFF769FC064605E082E0FFF764FC1C
:1020E000801B02287DD838688007F7D42078400705
:1020F00068D5DFF8CCB100270BF13C0BDBF8000012
:10210000C0000BD4DBF8001041F08051CBF8001078
:10211000DBF80000012700F0805000906B4E306823
:10212000C00510D4306840F480703060FFF73CFC8C
:10213000009005E0FFF738FC0099401A022850D8BB
:102140003068C005F6D55E4EA0686C3601280FD009
:102150000528306810D020F001003060306820F091
:1021600004003060A068B8B1FFF71EFC00900FE0DB
:10217000306840F00100F4E740F004003060F7E719
:10218000FFF712FC0099411A41F28830814266D86B
:1021900030688007F4D50EE0FFF706FC009007E0FA
:1021A000FFF702FC0099411A41F28830814256D86B
:1021B00030688007F4D42FB1DBF8001021F0805193
:1021C000CBF80010A069C8B33D49091D0968C1F3E7
:1021D000810102294AD00228504607D0C8F8600081
:1021E00000E03CE0FFF7E0FB04463BE04746C8F870
:1021F0006000FFF7D9FB064605E000BFFFF7D4FB00
:10220000801B02282BD828688001F7D4D4E9070165
:102210000843A16A2E4A490802EB0141626A41EA79
:102220008211084394F82C1040EA0161C9F80010AB
:1022300001203866FFF7B8FB044606E03EE000BF29
:10224000FFF7B2FB001B022809D828688001F7D5E8
:1022500034E000BFFFF7A8FB001B022802D90320CF
:10226000BDE8F88F28688001F4D427E00128F7D072
:10227000D9F80000E26900F4800191421CD1226A81
:1022800000F03F01914217D147F6C071626A0140E8
:10229000B1EB821F10D1A26A4FF0FF3300F440313E
:1022A00003EB5202B1EB024F06D194F82C1000F070
:1022B0007060B0EB016F01D00120D1E70020CFE7C3
:1022C0000438024000004742800E47420070004040
:1022D0000000FFFF70B5040009D0606A002540B11E
:1022E00025616561A56294F8510040B10CE00120C0
:1022F00070BD6068B0F5827FF4D0E561F2E784F8E4
:102300005050204600F044F8022084F85100206824
:10231000016821F040010160A088218900F48270E9
:1023200001F404410843A18901F400610843217CC0
:1023300001F002010843217D01F001010843218BD6
:1023400001F400710843217F01F03801084394F83B
:10235000201001F080010843218D01F40051084351
:1023600021680860A069042101EA104094F8241053
:1023700001F010010843216848602068C16921F418
:102380000061C1616565012084F85100002070BDC5
:102390002DE9F04387B0054614216846FEF7C3F8DF
:1023A000DFF81CC1296847480226012303270522BC
:1023B0000024614564D143491431D1F800C04CF484
:1023C000805CC1F800C0096801F480510591016882
:1023D00041F002010160016801F00201059101680C
:1023E00041F0010101600068984600F0010005908D
:1023F00018208DE84101CDE90372914669463248C3
:10240000FFF7D4F980208DE84101CDE903796946D1
:102410002E48FFF7CBF92F4E2D487F063060C6E9D6
:1024200001744FF48068C6E9034874614FF40030CA
:10243000B461C6E9074030467462FFF709F908B194
:10244000FEF7A1FCEE64B563224E214860361830D9
:10245000E6E802074020A6E81101800246F8144988
:10246000B461C6E907401B4874626030FFF7F0F8BA
:1024700008B1FEF788FCAE64B56307B0BDE8F08331
:10248000154CA142F9D10F4910310C6844F4804435
:102490000C60096801F480410591016841F4807184
:1024A00001600068029300F4807005900E20CDE971
:1024B0000006CDE9037269460848FFF777F9DCE7C3
:1024C0000030014030380240000402400000024069
:1024D00040640240C002002000380040002002405A
:1024E00010B5401EB0F1807F01D3012010BD4FF028
:1024F000E02460610F21601701F027FF0020A06138
:1025000007202061002010BD7047704770B590F81B
:102510003C20012A32D0012480F83C40022280F87D
:102520003D2003685A689D6822F070060A683243AD
:102530005A60134B02689A4214D0B2F1804F11D006
:10254000104B9A420ED0104B9A420BD00F4B9A422E
:1025500008D00F4B9A4205D00E4B9A4202D00E4B38
:102560009A4204D1496825F080031943916080F8AC
:102570003D40002180F83C10084670BD022070BD2F
:10258000000001400004004000080040000C004032
:1025900000040140004001400018004010B5040054
:1025A00003D094F83D0010B107E0012010BD0020D9
:1025B00084F83C00204600F01FF8022084F83D001B
:1025C000211D206801F0D4FA012084F8460084F827
:1025D0003E0084F83F0084F8400084F8410084F80D
:1025E000420084F8430084F8440084F8450084F8ED
:1025F0003D00002010BD000008B500681149884268
:1026000012D11148016841F02001016000680022E8
:1026100000F02000009005213720FFF787FBBDE880
:1026200008403720FFF774BB0849884209D10648A3
:10263000001D016841F400310160006800F40030C1
:10264000009008BD001400404038024000440140A2
:1026500070472DE9F04104460068C66805694FF0EF
:102660000007A90713D5B10711D5F91E0161012093
:102670002077206880698007204602D0FFF7E8FFB6
:1026800004E000F0A9F8204600F03BF9277768073E
:1026900016D5700714D521686FF004000861022078
:1026A00020772068806910F4407F204602D0FFF731
:1026B000CFFF04E000F090F8204600F022F92777E1
:1026C000280715D5300713D521686FF00800086179
:1026D000042020772068C0698007204602D0FFF7D9
:1026E000B7FF04E000F078F8204600F00AF92777F9
:1026F000E80616D5F00614D521686FF010000861C1
:10270000082020772068C06910F4407F204602D05E
:10271000FFF79EFF04E000F05FF8204600F0F1F8BC
:102720002777E80708D0F00706D021686FF001008E
:102730000861204600F0E6F8280608D5300606D5E0
:1027400021686FF0800008612046FFF7DDFE680613
:1027500008D5700606D521686FF040000861204654
:1027600000F0D1F8A8060AD5B00608D521686FF0A8
:10277000200008612046BDE8F041FFF7C6BEBDE875
:10278000F081000010B586B0044614216846FDF7BC
:10279000CAFE0E492068884215D10D480021026802
:1027A00042F020020260006800F020000590402006
:1027B00000900220CDE901010320CDE90310694614
:1027C0000448FEF7F3FF06B010BD000000440140CE
:1027D0003038024000140240704770B5044690F84B
:1027E0003C0000260D4601280FD0012084F83C0053
:1027F0006AB1042A1DD0082A2FD00C2A3FD0012606
:10280000002084F83C00304670BD022070BD206876
:1028100001F016FA2068816941F0080181612068A1
:10282000816921F004018161206881692A6911436D
:1028300011E0206801F034FA2068816941F40061F8
:1028400081612068816921F48061816120688169EA
:102850002A6941EA02218161D2E7206801F056FA33
:102860002068C16941F00801C1612068C16921F097
:102870000401C1612068C1692A69114311E020681F
:1028800001F078FA2068C16941F40061C1612068F3
:10289000C16921F48061C1612068C1692A6941EA86
:1028A0000221C161ACE710B5040003D094F83D00EB
:1028B00010B107E0012010BD002084F83C00204644
:1028C00000F01EF8022084F83D00211D206801F070
:1028D0004FF9012084F8460084F83E0084F83F0058
:1028E00084F8400084F8410084F8420084F84300F2
:1028F00084F8440084F8450084F83D00002010BDB1
:1029000070477047704770477047000010B501F07E
:1029100097FB03280AD000EBC001054800EB8100BB
:102920000069002802D0BDE81040004710BD00003B
:102930001C750020F8B5016804460868CA684B6930
:1029400010F00F0F4FF0000559D003F0010602F40C
:102950009077374365D0C10705D0D10503D5616CA9
:1029600041F001016164410705D5D90703D0616CCD
:1029700041F002016164810705D5D90703D0616C7C
:1029800041F004016164010707D502F020013143E1
:1029900003D0616C41F008016164616C00293AD098
:1029A000800604D5900602D5204601F05BFB206826
:1029B0004069616CC0F38010090700D460B3204601
:1029C00001F008FB20684069400621D520681430DA
:1029D00050E8001F21F0400140E80012002AF5D124
:1029E000E06BA8B172490165E06BFEF74EFD00286F
:1029F00011D0E06B016D01B0BDE8F04008478306DF
:102A00000FD593060DD52046BDE8F84001F02ABB4E
:102A10002046FFF77BFFF8BD2046FFF777FF656490
:102A2000F8BD266B2023012E7ED1C6067CD5D606A6
:102A30007AD508684868009048694FF00206400659
:102A40004DD5E26B106840684FF480770004000CAD
:102A50003AD0A18D814237D9E085D069B8422DD0D6
:102A600020680C3050E8001F21F4807140E800120B
:102A7000002AF5D12068143050E8001F21F0010130
:102A800040E80012002AF5D12068143050E8001FF9
:102A900021F0400140E80012002AF5D184F84230CC
:102AA000256320680C3050E8001F21F0100140E839
:102AB0000012002AF5D1E06BFEF79EFC6663A08D44
:102AC000E18D401A81B206E0A18D8142A8D1D06982
:102AD000B842A5D166632046FFF716FFF8BDA08D6A
:102AE000E18D401A81B2E08D0028F7D00029F5D0A1
:102AF00020680C3050E8002F22F4907240E8002744
:102B0000002FF5D12068143050E8002F22F0010288
:102B100040E80027002FF5D184F842302563206873
:102B20000C3050E8002F00E006E022F0100240E8F0
:102B30000023002BF3D1CDE705062BD5150629D5AB
:102B400094F841002128C9D1A068B0F5805F01D177
:102B50002069B0B1206A411C216221680078486078
:102B6000E08C401E0004000CE084B7D12068C168EE
:102B700021F08001C1602068C16841F04001C1605E
:102B8000F8BD206A0088C0F308004860206A801CF5
:102B90002062E5E74006F3D55006F1D5CA68204625
:102BA00022F04002CA6084F8413000F01DFAF8BDFE
:102BB000D93E000870B5040004D094F84100002507
:102BC00010B106E0012070BD84F84050204600F0AE
:102BD00023F8242084F841002068C16821F40051C2
:102BE000C160204601F0A0FA2068016921F49041FB
:102BF00001612068416921F02A0141612068C168B2
:102C000041F40051C1606564202084F8410084F8DB
:102C100042006563002070BD2DE9F04F87B0054686
:102C200014216846FDF77FFCC648DFF8148314388A
:102C30000221D5F800C0DFF80CA3032207238F067A
:102C4000002406154FF04009C44576D1DAF800801B
:102C500048F01008CAF80080DAF800C00CF0100C38
:102C6000CDF814C0D0F800C04CF0020CC0F800C081
:102C7000D0F800C00CF0020CCDF814C0D0F800C0A1
:102C80004CF0010CC0F800C00068884600F001005C
:102C900005908020CDE90008CDE9024293469A468E
:102CA00069460493A848FEF781FD7010CDE900083D
:102CB000CDE9024B6946CDF810A0A448FEF776FD99
:102CC000DFF89082A2494046C8F80010C0E90174BC
:102CD000C0E90346C8F81440C8F81840C8F81C40BA
:102CE000C8F82040BA46C8F82440FEF7B1FC08B145
:102CF000FEF749F8974FC5F83C806037C8F8385060
:102D0000C7F80890C7E903467C61BC619048FC6144
:102D10003C6230307C62C7E9000A3846FEF798FC16
:102D200008B1FEF730F8AF63002205212520BD630E
:102D3000FEF7FCFF2520AAE0FFE7DFF81C82DFF8A2
:102D400004B2C445ABF1040B57D1DBF8008048F462
:102D50000038CBF80080DBF800C00CF4003CCDF864
:102D600014C0D0F800C04CF0080CC0F800C00068D7
:102D700000F00800059060208DE813006946774850
:102D8000CDE90323FEF712FDDFF8C881744908F18D
:102D9000C0084046C8F80010C0E90174C0E9034605
:102DA000C8F81440C8F81840C8F81C40C8F82040BB
:102DB000BA46C8F82440FEF74BFC08B1FDF7E3FF24
:102DC000684FC5F83C80C8F83850C7F80890C7E984
:102DD00003467C61BC616248FC613C6218307C62E5
:102DE000C7E9000A3846FEF733FC08B1FDF7CBFF10
:102DF000AF63BD6307B0BDE8F08FDFF86C81C445F9
:102E000048D1DBF8008048F48028CBF80080DBF85C
:102E100000C00CF4802CCDF814C0D0F800C04CF0E9
:102E2000040CC0F800C0006800F0040005904FF4E6
:102E300040608DE8130069464C48CDE90323FEF756
:102E4000B5FCDFF82081464908F16008603940464A
:102E5000C8F80010C0E90174C0E90346C8F814407E
:102E60004FF40031C8F81840C8E90741C8F82440B9
:102E7000FEF7EEFB08B1FDF786FFC5F83C800022A7
:102E800005212720C8F83850FEF750FF2720FEF70D
:102E90003FFFAFE7364B9C45ACD1DAF8007047F006
:102EA0002007CAF80070DAF8003003F02003059319
:102EB000036843F040030360006800F040000590A1
:102EC0004FF484408DE813000820CDE903206946C3
:102ED0002848FEF76BFC234F1D48C0376038386028
:102EE0004FF02068C7E90184C7E903467C614FF4CD
:102EF000803ABC61C7E9074A38467C62FEF7A8FB06
:102F000008B1FDF740FFEF63BD631B4F1048C7E9F1
:102F100003467C61BC61C7E9074A18307C6287E8D8
:102F200001033846FEF794FB08B1FDF72CFFAF63B1
:102F3000002205214720BD63FEF7F8FE4720A6E7E3
:102F400000100140443802400004024000000240EA
:102F5000886402403005002000440040000C02401C
:102F600088600240500600200048004000080240EF
:102F700000140140001802407007002090F8423011
:102F8000202B01D00220704721B11AB10023036326
:102F900001F050B90120704710B501F051F8032835
:102FA0000AD000EBC001054800EB8100C068002892
:102FB00002D0BDE81040004710BD00001C75002085
:102FC00010B501F03DF803280AD000EBC001054818
:102FD00000EB81008068002802D0BDE81040004767
:102FE00010BD00001C75002010B501F029F8032861
:102FF0000AD000EBC001054800EB810040680028C2
:1030000002D0BDE81040004710BD00001C75002034
:10301000FEE7000038B390ED061AD0ED011AF0EE8D
:10302000400A90ED022A41EE610AD0ED071A4FF0F6
:103030007F4241EEC20A10EE901AB2EB410F01D16D
:10304000F0EE400A90ED040A90ED032A21EE000A0A
:1030500000EE820A90ED052A80ED071AC0ED060AFF
:1030600001EE820A70479FED010A704700000000E0
:10307000B8B1D0ED030A90ED041A70EE810A90ED1C
:10308000051A30EE811AC0EE010A10EE901A6FEAAE
:10309000D15111F0FF0F07D0C0ED060AC0ED070AAD
:1030A00006E09FED040A704780ED060A80ED070AEE
:1030B000FFF7B0BF0000000010B190ED050A7047A7
:1030C000B8EE000A70470000022801D300207047C4
:1030D000014951F820007047A800002030B10128B4
:1030E00007D0022808D04FF0FF30704742F210702E
:1030F00070474FF48040704747F23050704770B5CA
:10310000040015D02078FFF7DFFF00280CD0002145
:1031100090F844300AE000EB810292692AB15588A8
:103120006688B54201D1104670BD491C8B42F2DC65
:10313000002070BD70B504002DED028BB0EE408A0A
:103140000ED02078FFF7C0FF05006FF0030625D0F2
:1031500018EE100AB0F17E5F07DDB7EE008A0BE0D3
:103160006FF00100BDEC028B70BD18EE100A10F17B
:10317000814F01D9BFEE008A607908B1B1EE488A6B
:103180002046FFF7BCFF48B1618820794FF0FF323D
:1031900030B1012804D0022810D109E03046E1E71F
:1031A000A1F20121072909D24CB2002C06DB07E06D
:1031B000A1F20523062B01D2491EF5E71046D1E7FF
:1031C000AD1CFFF78BFF00EE100AB8EEC00A20EE30
:1031D000080ABDEEC00A10EE100A25F814000020FF
:1031E000C0E700000F4810B50D49016003214160A0
:1031F00000214FF410228160C0E903124FF4001245
:103200004261017641768176C17601774177FDF79B
:10321000D1FE002803D0BDE81040FDF7B4BD10BDBD
:1032200000640040C40000200F4810B50D49016043
:103230000321416000214FF410228160C0E9031294
:103240004FF400124261017641768176C1760177B2
:103250004177FDF7AFFE002803D0BDE81040FDF731
:1032600092BD10BD00680040EC0000202D4808B55C
:10327000016841F480010160016801F4800100915E
:10328000016841F4001101600068002200F40010A0
:10329000009005210C20FEF749FD0C20FEF738FDBB
:1032A000002205211020FEF741FD1020FEF730FD21
:1032B000002205211120FEF739FD1120FEF728FD1F
:1032C000002205213920FEF731FD3920FEF720FDCF
:1032D000002205213A20FEF729FD3A20FEF718FDCD
:1032E000002205213B20FEF721FD3B20FEF710FDCB
:1032F000002205214420FEF719FD4420FEF708FDB9
:10330000002205214520FEF711FD4520FEF700FDB6
:10331000002205214620FEF709FDBDE808404620B1
:10332000FEF7F6BC3038024010B5074A00210748C6
:1033300001F022FC0649074A0860BDE81040002160
:10334000054801F019BC0000246E0008993A0008F5
:1033500000000020686E0008C53D00082DE9F0431C
:1033600087B014216846FDF7DEF84F48016841F048
:1033700002010160016801F002010591016841F05C
:1033800040010160016801F040010591016841F0D0
:1033900001010160016801F001010591016841F03E
:1033A00008010160016801F008010591016841F020
:1033B00004010160016801F004010591016841F414
:1033C00080710160016801F480710591016841F02C
:1033D00020010160016801F020010591016841F0C0
:1033E000800101600068314F00F0800005900022EC
:1033F00040213846FEF7D2FADFF8B48001221021CE
:103400004046FEF7CBFADFF8AC9041F2010601220C
:1034100031464846FEF7C2FA01244020CDE90004B7
:103420000294694638460394FEF7C0F908204FF429
:103430000415CDE90005694602943846FEF7B6F951
:103440001020CDE900040294694640460394FEF73B
:10345000ADF93020CDE90005694602941648FEF723
:10346000A5F9CDE900640294694648460394FEF745
:103470009DF9002205210920FEF758FC0920FEF7DE
:1034800047FC002205210A20FEF750FC0A20FEF727
:103490003FFC002205211720FEF748FC1720FEF70D
:1034A00037FC07B0BDE8F083303802400018024016
:1034B0000000024000040240000802400D4810B520
:1034C0000B4901600C49416000214FF4804281604A
:1034D000C0E9031241618161C1610162FEF76AFACC
:1034E000002803D0BDE81040FDF74DBC10BD000022
:1034F0000054004014010020801A06000D4810B549
:103500000B4901600C49416000214FF48042816009
:10351000C0E9031241618161C1610162FEF74AFAAB
:10352000002803D0BDE81040FDF72DBC10BD000001
:103530000058004068010020A08601000D4810B529
:103540000B4901600C49416000214FF480428160C9
:10355000C0E9031241618161C1610162FEF72AFA8B
:10356000002803D0BDE81040FDF70DBC10BD0000E1
:10357000005C0040BC010020A0860100104810B58E
:103580000E4901604FF48271416000210222816086
:10359000C0E9031201224261520282611822C0E98D
:1035A0000721416281620A21C162FEF793FE002871
:1035B00003D0BDE81040FDF7E6BB10BD0030014070
:1035C00010020020104810B50E4901604FF48271BE
:1035D000416000218160C1604FF400720161C0E967
:1035E00005122822C0E90721416281620A21C162D5
:1035F000FEF770FE002803D0BDE81040FDF7C3BB06
:1036000010BD0000003800406802002010B588B0EE
:103610001C216846FCF787FF144813490024C0E9C1
:10362000001441F28731C0E9024104618461FEF770
:10363000B5FF08B1FDF7A7FB0C48FFF734F908B157
:10364000FDF7A1FB6020CDE9000402940022694649
:1036500006480494FFF7C1F808B1FDF794FB03484E
:10366000FFF790F808B010BD00440140C8030020E7
:103670001CB500240E4800940C490194C0E90014C4
:1036800040F2E731C0E902418461FEF787FF08B1EB
:10369000FDF779FB0094694605480194FEF736FF73
:1036A000002801D0FDF76FFB1CBD00000014004096
:1036B000800300200C4810B50A4901604FF4E13145
:1036C0004160002181600C22C160C0E90412816167
:1036D000C161FFF76FFA002803D0BDE81040FDF785
:1036E00052BB10BD00100140100400200C4810B562
:1036F0000A4901604FF4E1314160002181600C22F0
:10370000C160C0E904128161C161FFF753FA00286A
:1037100003D0BDE81040FDF736BB10BD00440040AB
:10372000580400200D4810B50B4901600C49416058
:1037300000214FF480628160C0E903120C22C0E9CD
:103740000521C161FFF736FA002803D0BDE810401B
:10375000FDF719BB10BD000000480040A004002088
:10376000A08601000C4810B50A4901604FF4E13110
:103770004160002181600C22C160C0E904128161B6
:10378000C161FFF717FA002803D0BDE81040FDF72C
:10379000FABA10BD00140140E8040020FEE7000062
:1037A00030B54FF0FF3400287ED00078DFED540AAA
:1037B000062834D2DFE800F003354C5B5B59042B5C
:1037C00055D191EC021A31EE611AD1ED021A31EEA7
:1037D000211A82ED001A91EC021A31EE211AD1ED74
:1037E000021A31EE211A82ED011A91ED011AD1ED82
:1037F000001A31EE611AD1ED021A31EE211A82ED72
:10380000021A91ED001AD1ED011AB1EE411A31EE12
:10381000611AD1ED021A31EE211A82ED031A00204D
:103820003DE0042B23D191ED000AB1EE400A82ED78
:10383000000A91ED000A82ED010A91ED000A82ED85
:10384000020A91ED000AB1EE400A82ED030A0EE091
:10385000022B0CD191ED000AB1EE400A82ED000A74
:1038600091ED000A82ED010A07E0012B01D0002052
:1038700042E091ED000A82ED000A002036E000BF30
:1038800002EB800191ED001AB0EEC11AB4EEE01A1D
:10389000F1EE10FA01DDF0EE410A401C40B2984210
:1038A000EEDB10EE900A00E028E0B0F17E5F0DDD67
:1038B000002009E002EB8001401C91ED001A40B2AB
:1038C000C1EE201AC1ED001A9842F3DB002009E096
:1038D00002EB8001401CD1ED000A40B260EE800A8C
:1038E000C1ED000A9842F3DB002030BD02EB8001FD
:1038F000401CC1ED000AC0B29842F7DB204630BD43
:1039000000000000FEE7000010B504462DED068B18
:10391000B0EE409AF0EE618AB0EE418AF0EE609A25
:1039200019EE100A00F00AFD002850D019EE900A96
:1039300000F004FD00284AD0B0EE480A10EE100A4C
:1039400000F0FCFC002842D018EE900A00F0F6FCD3
:10395000E8B36068F0EE690AB0EE490A90ED071A24
:10396000FDF714F96068B0EE409AD0ED000A04F15A
:103970001C0020EE89AA20EEA90AFFF74BFB207855
:10398000DFED38AAF0EE409A70B101280ED1D4EDE7
:10399000020AB0EE680A00F091FDD4ED050A79EE56
:1039A000E00A80EE808A01E0B0EE6A8A18EE100A22
:1039B00084ED049AC4ED059A6FEAD05010F0FF0F21
:1039C00001D1B0EE6A8A606890ED010A00E045E03E
:1039D00020EE0A0AD0ED030AD0ED021A224A08EEC0
:1039E000600AD4ED030A11EE901A4AEE280A9142B9
:1039F00021EEA01A1CDD10EE901A6FEAD15111F0E1
:103A0000FF0F15D070EE011A90ED052AF0EEE11AC5
:103A1000F4EEC21AF1EE10FA0AD890ED042AF0EE94
:103A2000E01AF4EEC21AF1EE10FA01D8C4ED030A5E
:103A300030EE010A10EE101A6FEAD15111F0FF0FAB
:103A40000CD0D0ED050A10EE900A904201DDFCF793
:103A500030FE84ED060ABDEC068B10BD94ED060A1F
:103A6000F9E7000000000000BD37863510B570B1E1
:103A70009FED080A80ED030A80ED040A80ED050A37
:103A800080ED060A1C30FFF7F3FA002010BD4FF05E
:103A9000FF3010BD0000000010B501F06AF8BDE86D
:103AA000104001F0AEB810B5FEF7D4F802F03CFCBF
:103AB000012803D0BDE8104002F052B810BD00004C
:103AC00030B593B030216846FCF72DFD14210CA8C9
:103AD000FCF729FD1D480025016841F08051016077
:103AE000006800F0805011901948016841F480414D
:103AF00001600068022400F48040119001200090D1
:103B0000000401908001CDE9064006200890A8201D
:103B1000CDE9090404200B906846FEF725FA08B1A8
:103B200072B6FEE70CA90F2081E831004FF4A050D7
:103B30000F904FF48050109005210CA8FEF728F943
:103B4000002801D072B6FEE713B030BD4038024005
:103B5000007000400248016841F470010160704744
:103B600088ED00E00148FEF774BD000080030020EE
:103B7000F0B50268274B284D284E294F294C4FF0AD
:103B8000804C984209D0604507D0A84205D0B04289
:103B900003D0B84201D0A04204D122F0700E4A688E
:103BA00042EA0E0298421BD0604519D0A84217D0B5
:103BB000B04215D0B84213D0A04211D01A4DA8423D
:103BC0000ED01A4DA8420BD0194DA84208D0194D5D
:103BD000A84205D0184DA84202D0184DA84203D1E2
:103BE00022F44075CA682A434D6922F080022A43B4
:103BF0008D68C5620D688562984201D0A04201D1EE
:103C000009690163016841F004010160012141611A
:103C10000260F0BD000001400004004000080040C8
:103C2000000C0040000401400040014000440140FD
:103C30000048014000180040001C004000200040E7
:103C4000F0B5036A026A22F00102026242688469E6
:103C5000124E24F073050C682C4323F002058B6888
:103C60002B430D4DA84201D0B04205D123F00807E7
:103C7000CB683B4323F00403A84201D0B04205D1F6
:103C80004D6922F4407215438A692A434260846177
:103C9000496841630362F0BD000001400004014037
:103CA000F0B5026A036A23F0100303624368846973
:103CB0000D6824F4E64444EA05248D6822F02002CD
:103CC00042EA05120F4D104EA84201D0B04206D173
:103CD000CF6822F0800242EA071222F04002A84296
:103CE00001D0B04207D14D6923F4406343EA850314
:103CF0008D6943EA85034360846149688163026298
:103D0000F0BD00000000014000040140F0B5026A6F
:103D1000036A23F4807303624368C46922F4007267
:103D200024F073050C68124E2C438D6842EA05227C
:103D30000E4DA84201D0B04206D1CF6822F40062F5
:103D400042EA072222F48062A84201D0B04207D1A1
:103D50004D6923F4405343EA05138D6943EA051383
:103D60004360C4614968C1630262F0BD0000014064
:103D70000004014030B5046A026A22F480520262F3
:103D80004268C3690D6823F4E64343EA05238D685E
:103D900024F4005444EA0534084DA84202D0084DEA
:103DA000A84204D14D6922F4804242EA8512426061
:103DB000C36149680164046230BD00000000014035
:103DC0000004014010B500F0D3FD0A4A00210A4862
:103DD00000F0D2FE094C00220A212060022000F0EF
:103DE00016FE606000F0F6FD00F0C3FEBDE8104076
:103DF00000F007BF8C6E0008013E000864750020CB
:103E000000F0A1FD02F04BFE9FED2C1B53EC112B9B
:103E100002F0C0FC02F016FE0546002000F068FD2E
:103E200000F08AFD04462748FCF756FF2C4425483D
:103E3000FCF786FF1420FCF792FFB0B32249A1F1F2
:103E4000A000FCF759FE2048022110389FED1F0A00
:103E500001701C49D1ED0A0A30EEC01ADFED1C0AD0
:103E600021EE201A80ED011A91ED091A31EE401A67
:103E700061EE200AC0ED020AD1ED0B0A30EEC00A55
:103E8000DFED140A20EE200A80ED030A00F054FD55
:103E90000D4902461039A1F19000FCF791FC0A4946
:103EA000A1F1A000FCF7C2FD03E0FFE70548FCF725
:103EB00031FF204600F029FDB8E7000000000000B7
:103EC00000407F40187900202876002000008044C0
:103ED0006F12033B6F12833A10B5806B0021C185CE
:103EE000FEF714FD10BD70B5846B2068406994F82E
:103EF0004110C0F3C0100025212904D118B1E58478
:103F0000204600F08EF82068406994F84210C0F313
:103F10008010222904D118B1E585204600F05AF816
:103F2000606C40F0100060642046FEF7EFFC70BD4E
:103F300010B50146806B096809684FF00002C90599
:103F40002ED4C28501680C3151E8003F23F4807300
:103F500041E80034002CF5D10168143151E8003FEC
:103F600023F0010341E80034002CF5D1016814313D
:103F700051E8003F23F0400341E80034002CF5D124
:103F8000202180F84210016B012909D101680C3110
:103F900051E8003F23F0100341E80034002CF5D134
:103FA0004263016B012902D0FEF7F6FF10BD818D3F
:103FB000FEF7AAFC10BD10B5806B01214163016BB7
:103FC000012902D0FEF7FCFF10BD818D4908FEF7E4
:103FD0009BFC10BD01680C3151E8002F22F4907257
:103FE00041E80023002BF5D10168143151E8002F7E
:103FF00022F0010241E80023002BF5D1016B0129D9
:1040000009D101680C3151E8002F22F0100241E87B
:104010000023002BF5D1202180F8421000210163FC
:10402000704701680C3151E8002F22F0C00241E8CE
:104030000023002BF5D1202180F8411070470000AB
:1040400000680649884201D100207047044988422F
:1040500001D101207047032070470000001001408B
:104060000048004008B590F84210222901D00220F3
:1040700008BD82684FF480539A4201D1016921B191
:10408000816A9A421BD04AB10AE00268816A52688A
:10409000C2F308020A80816A891C08E0026972B1D1
:1040A0000268526802F07F020A70816A491C8162CC
:1040B000C18D491E0904090CC18503D01BE00268AB
:1040C0005268F1E70168CA6822F02002CA600168FC
:1040D000CA6822F48072CA6001684A6922F001024B
:1040E0004A61202180F8421000214163026B012ABD
:1040F00003D0FEF751FF002008BD016301680C31B9
:1041000051E8002F22F0100241E80023002BF5D1E6
:1041100001680A68D20602D50A6849680091818D53
:10412000FEF7F2FBE7E7000070B50446006801699E
:10413000E26821F44051114301612169A068E269FC
:1041400008436169114308432168CA6849F20C6356
:104150009A430243CA6020684169A26921F4407110
:104160001143416131492068884202D03049884278
:1041700002D1FDF7B7FE01E0FDF7A4FEE2690023DE
:10418000192164253226B2F5004F626828D0A0FBC1
:104190000101930F9200FCF7E3F80146B0FBF5F044
:1041A0006FF01802504301EB800006EB0010B0FBEB
:1041B000F5F000F0F002B1FBF5F002EB0012B1FBFC
:1041C000F5F06FF01803584301EB800006EB001088
:1041D000B0FBF5F000F00F0021681044886070BD5E
:1041E000A0FB010192185B41FCF7BAF80146B0FB55
:1041F000F5F00201B1FBF5F06FF01803584301EB45
:10420000800006EBC000B0FBF5F000F0F80002EB18
:104210004002B1FBF5F0584301EB800006EBC00013
:10422000B0FBF5F000F00700D6E7000000100140F9
:104230000014014038B5816204468285002013468F
:104240006064222284F84220E56B1F4AEA63E56B32
:104250001E4A2A64E56B1E4AEA64E26B10650A4650
:104260002168E06B091DFDF75DFA30B11020606434
:10427000202084F84200012038BD20680168406891
:104280000090206948B120680C3050E8001F41F4CC
:10429000807140E80012002AF5D12068143050E8FF
:1042A000001F41F0010140E80012002AF5D120680A
:1042B000143050E8001F41F0400140E80012002A8D
:1042C000F5D1002038BD0000313F0008B73F00089D
:1042D000E73E000810B50448FEF72CFBBDE810408F
:1042E0000148FCF707BA00001004002010B5FFF7E2
:1042F000FDFF0448FEF71EFBBDE810400148FCF737
:10430000F9B90000A00400200148FEF713BB00002B
:10431000E8040020FEE74100080218BF04200A0E4E
:1043200018BF40F001004FF07F4232EA010108BFA0
:1043300040F00200012808BF052070476FEAD05006
:1043400010F0FF0000D0012070470907090E002877
:1043500004DB00F1E02080F80014704700F00F004B
:1043600000F1E02080F8141D7047000010EE101AD4
:1043700008B5444A6846B2EB410F28D94FF0E640F1
:10438000B0EB410F94BF00204FF0FF300090009839
:10439000002861DB60EE000A10F0010F45D010F03C
:1043A000020FDFED391A9FED391A00EEE11ADFED49
:1043B000381A40EE811A21EEA01AF0EE400A40EEC3
:1043C000010A08BFF1EE600AB0EE600A08BD314B89
:1043D00021F0004293423CD911F0004FDFED2E0A4C
:1043E00020EE201ADFED2D0A19BF31EE601A71EEB2
:1043F000200A31EE201A71EE600ABDEEE01A11EECD
:10440000100A9FED271A00F0030000EEC10A9FED8D
:10441000251A009000EEC10A9FED231A00EEC10A92
:104420009FED221A00EEC10AB1E79FED211A9FED20
:10443000210A10F0020F00EE810A9FED1F1A00EE14
:10444000801AB7EE000A00EE810A18BFB1EE400AEA
:1044500008BD00F033F99AE710EE100A4000B0F101
:104460007F4F3CBFB7EE000A08BD07D14FF00100F7
:10447000FCF788F8BDE8084000F010B9BDE8084036
:1044800000F008B9B61F927E336D4C39DA82083CD1
:10449000A0AA2ABE490E494683F9223F0000004BDC
:1044A0000000C93F00A0FD390020A2331A61342C5E
:1044B000B93AB2BACA9F2A3DDDFFFFBE10B52DED55
:1044C000028BB0EE608AF0EE408A18EE101A18EEF9
:1044D000900A02F02DFC00F07040B0F1005F0CD0AB
:1044E00018EE100A20F00040C0F1FF40C00F02BFDC
:1044F000B0EE480ABDEC028B10BDB0EE680ABDEC10
:10450000028B10BD00B510EE101A2DED028B81B09C
:10451000524A6846B2EB410F2ED94FF0E640B0EB5D
:10452000410F94BF00204FF0FF3000900098B0EE94
:10453000408A00286ADB10F0010F4BD068EE080AB1
:104540009FED471A9FED470A00EE810A9FED461A3C
:1045500010F0020F00EE801AB7EE000A00EE810A9A
:1045600002BF01B0BDEC028B00BD00BF01B0B1EED7
:10457000400ABDEC028B00BD3C4B21F0004293424F
:1045800041D911F0004FDFED3A0A20EE201ADFED9D
:10459000390A19BF31EE601A71EE200A31EE201A85
:1045A00071EE600ABDEEE01A11EE100A9FED321AAC
:1045B00000F0030000EEC10A9FED301A009000EEFB
:1045C000C10A9FED2F1A00EEC10A9FED2E1A00EED0
:1045D000C10AABE728EE080A9FED2B1ADFED2B0A84
:1045E00010F0020F40EE410A9FED291A00EE201A4A
:1045F00061EE000AB0EE480A08EE200AB6D101B01A
:10460000BDEC028B00BD00F059F88FE718EE100AE0
:104610004000B0F17F4F0DD218EE100AFFF77BFE7D
:10462000042808BF00F042F8B0EE480A01B0BDEC23
:10463000028B00BD09D10120FBF7A4FF01B0BDEC46
:10464000028B5DF804EB00F029B801B0B0EE480A27
:10465000BDEC028B5DF804EB00F01CB8B61F927E37
:10466000B93AB2BACA9F2A3DDDFFFFBE490E49469C
:1046700083F9223F0000004B0000C93F00A0FD3934
:104680000020A2331A61342C336D4C39DA82083C95
:10469000A0AA2ABE30EE000A70470000DFED020A31
:1046A00080EEA00A70470000000000009FED020AA3
:1046B00020EE000A70470000000000102DE9F00114
:1046C0004FF07F42B2EB410F9FBF4FF0FF310160CF
:1046D000BDE8F00170474FF0004242EA0123C1F308
:1046E000C752783A551112F01F0C434CCCF12006FA
:1046F0007C44C1F3C752A2F178024FEA621204EB84
:10470000820254F8254008BFD2E9015612D05568FC
:1047100004FA0CF425FA06F73C43976805FA0CF501
:1047200027FA06F8D26807FA0CFCF24045EA0805B9
:104730004CEA0206A4FB034CA5FB0352A6FB036351
:104740001D449D4234BF012600261319334416B17F
:10475000934202D903E0934201D2012200E00022F9
:10476000624402F1200C9206DC0C42EA443200EE74
:10477000102A5B03DFED210AF8EEC01A00EE103AB2
:104780004FEA9C1C11F0004FB8EE400AC0F800C080
:1047900020EE201A00EE105ADFED190AB8EE400A9A
:1047A00020EE200A71EE810A70EE800A10EE902A47
:1047B00002F500626FF30B0200EE902A70EEE11A30
:1047C00031EEC11ADFED101A30EE411A9FED0D0ADD
:1047D00020EE800A01EE210A9FED0C1A00EE810AFC
:1047E00004BFBDE8F0017047CCF180510160BDE825
:1047F000F001B1EE400A7047BC270000000000360F
:104800000000802C22AAFD29DB0FC92F0000C92F30
:10481000704700002DE9F041040006D0184E3068C2
:1048200084420AD10020BDE8F081502080F3118835
:10483000BFF34F8FBFF36F8FFEE700F0A9FE6569EE
:10484000F76B366C00F0C4FEBD4201D0B54201D119
:104850000220E8E70B48854208D1A06A0028F7D17A
:1048600094F860000128F3D00320DCE705481438F1
:10487000854202D00DB10120D5E70420D3E7000026
:1048800018000020C00C002000207047FDF7EAF956
:10489000FFF716F9FEF762FDFEF7E8FCFEF7A2FC53
:1048A000FEF7C2FCFEF70AFEFEF728FEFEF746FE04
:1048B000FEF764FEFEF786FEFEF7FCFEFEF732FF13
:1048C000FEF750FFFEF7A2FEFEF710FFFEF7D0FE48
:1048D000122205490548FEF751FB00F037F8FEF7B4
:1048E00023FD00F05BF8FEE7B0000020A0040020EC
:1048F00010B5EFF3058111B16FF0050403E000245A
:1049000008B100F01DFF204610BD38B50546EFF395
:10491000058010B16FF005040CE0002401F012FDD9
:10492000291A0090002903DD684600F02FFF01E0FE
:104930006FF00304204638BDEFF3058008B101F0A5
:1049400007BD01F0FFBC4FF47A707047EFF30580AC
:1049500010B16FF0050070470448016811B14FF0C5
:10496000FF30704701210160002070477000002077
:1049700010B5EFF3058010B16FF0050010BD01F028
:10498000D3FC20B1022804D04FF0FF3010BD01202D
:1049900010BD01F011F8002010BD000010B5EFF3BC
:1049A000058010B16FF0050010BD084801680129AD
:1049B00002D04FF0FF3010BD054A002182F8141DCF
:1049C0000221016000F0B2FF002010BD7000002045
:1049D0000BE000E070B5EFF3058010B16FF0050457
:1049E00013E001F0A1FC4FF0FF3510B102280BD10C
:1049F00008E0012401F0D6FD012806D001F094FC66
:104A000010B102E0002400E02C46204670BDF8B54D
:104A100014464FF00005EFF3058212BB08B301B353
:104A2000A4B1D4E9023263B1502A1AD32269C2B1C7
:104A3000676900FB01F6B74213D3009501F0C7F890
:104A400007E072B9226962B9626952B9002201F0C5
:104A50009DF8050005D00CB1216800E0002100F0B0
:104A600039FE2846F8BD00003EB5040001D00029FB
:104A700003DA6FF0030001902BE04FF0FF3001905C
:104A8000EFF30580D0B1002502A800902B4601224B
:104A90000295204601F0C0FB002201AB11462046E2
:104AA000009501F0B9FB029898B10B494FF0805086
:104AB0000860BFF34F8FBFF36F8F0AE0002301221E
:104AC000204601F039FB002201AB1146204601F0DF
:104AD00033FB01983EBD000004ED00E02DE9F84FE6
:104AE000894605464FEA0206EFF3058010B16FF0E4
:104AF00005041EE0002D02DA6FF0030419E05FEAFE
:104B0000897002D54FF0000800E0A84600249246C4
:104B100001F018FC8346E71E53466A4641460020D2
:104B200001F082FC012807D00EB36FF001040028C9
:104B3000F2D12046BDE8F88F00982C4004435FEA8C
:104B4000C9700BD035EA0400F3D056B101F0FAFB7E
:104B5000A0EB0B00504506D9002006E02542E8D125
:104B6000F3E73C46E5E7AAEB00008246D4E73C4683
:104B7000DDE701F0D3BB00002DE9FF414FEA01035F
:104B80004FF00005EFF30581039549BB40B3802743
:104B9000182100244AB3166806B1344696691EB13E
:104BA0003146761E382E02D21679F60703D0002041
:104BB00004B0BDE8F081566906B1B708D2F808C064
:104BC000BCF1000F0DD0D568642D18D312693AB12D
:104BD00036B18DE806103A46214601F082FA03907C
:104BE0000DE0D6685EB912694AB903AACDE9001290
:104BF000BAB2214601F048FA012800D00395039883
:104C0000D6E770B50546EFF3058010B16FF00504E7
:104C10000FE04DB12846FFF7FDFD042807D0002422
:104C2000284600F0F9FD04E06FF0030401E06FF0A6
:104C30000204204670BD00002DE9F041134C0F46E0
:104C40000546E6682068001D00F044FC681C07D19A
:104C500037B12168BDE8F0410D48091D00F08BBC5B
:104C600020683544B5424560216805D2206CBDE816
:104C7000F041091D00F067BCE06B091D00F063FC0A
:104C8000A06A854200D2A562BDE8F081180000202C
:104C9000C00C00202DE9F041054600F079FC2D4CB8
:104CA000A068401CA06020682B4F10B1606930B331
:104CB0002BE02560A068012827D1002606EB86009E
:104CC00007EB800000F031FC761C382EF6D3234829
:104CD00000F02BFC2148143000F027FC1F4828303E
:104CE00000F023FC1D483C3000F01FFC1B485030F6
:104CF00000F01BFC1948E0631430206405E02068D4
:104D0000E96AC06A884200D82560606A401C606217
:104D1000A864E86A2169884200D9206100EB80001C
:104D200007EB8000291D00F026FC00F051FC6069B3
:104D300000280CD02068E96AC06A884207D2084976
:104D40004FF080500860BFF34F8FBFF36F8FBDE807
:104D5000F08100001800002010080020700C0020D6
:104D600004ED00E038B500F013FC104C2068C8B921
:104D70000F4800F0DAFB0E48143000F0D6FB0C4868
:104D8000E060143020610A4B0020F03B009003F1FA
:104D9000500210210A2000F01AFF206010B105A176
:104DA00000F098FCBDE8384000F012BC5C00002028
:104DB000C40D0020546D72510000000030B4026C2C
:104DC0000B46002A0BD0C1681144C1608468A1421F
:104DD00001D30168C16030BC1846FBF757BB30BC3B
:104DE00070472DE9F041856B174604460026026C9A
:104DF00082B1C7B1E068FBF749FBE168206C091A92
:104E0000E1602268914202D2A168081AE060022F94
:104E100016D017E02068A8B9A06801F04BFB064641
:104E20000020A0600EE06068FBF730FB216C60683A
:104E300008446060A168884204D32068606001E093
:104E400005B16D1E6D1CA5633046BDE8F08110B53F
:104E5000044690F8610058B101280CD002280FD008
:104E6000502080F31188BFF34F8FBFF36F8FFEE7A1
:104E7000206B00F0C1FB2046BDE8104000F0BCBB39
:104E800010BD000010484FF4C041420706D0C01DBD
:104E90000D4920F00700411AC1F5C0410B4A00231B
:104EA0000144C2E900030839183A21F007011160F2
:104EB0004B600B600B1AC0E9001393604FF0004089
:104EC0005360506170470000B41400208C00002033
:104ED000144E154CA6F29C474FF08058DFF84C90CA
:104EE00012E000BF00F054FBF068C568281D00F018
:104EF000F1FAA068401EA0606068401E606000F08B
:104F000067FB2846FFF7A3FF60680028EAD13868EE
:104F10000128F9D9C9F80080BFF34F8FBFF36F8F15
:104F2000F2E70000AC0C00201800002004ED00E0C7
:104F300070B51D46049C51B1C4F80020C4E90F01AE
:104F40000121204600F076FE84F84C5070BD2460AC
:104F5000F4E72DE9F05F8846DDE90B9415468346BA
:104F600091009A460A9EA522206BFBF7D4FA6FF0B7
:104F70000301206B01EB8501084420F00707780747
:104F800007D0502080F31188BFF34F8FBFF36F8F8E
:104F9000FEE700256764B8F1000F0ED0002022184C
:104FA00018F8001082F8341018F8001011B1401CE5
:104FB0001028F4D384F8435001E084F83450382E9C
:104FC00000D33726E662C4E91465201D00F0B8FA64
:104FD00004F1180000F0B4FA2461C6F138006462EC
:104FE000A061A565E56584F860505246594638468B
:104FF00000F05AFA2060B9F1000F01D0C9F8004062
:10500000BDE8F09F30B5114900E011460A688242C0
:10501000FBD34B685C18844203D140681844486055
:10502000084643681C18944209D1084C183C24686F
:10503000A24209D052681A4442600A6812680260AB
:10504000814200D0086030BD0460F9E78C00002088
:1050500070B5002441600B4D0061914206D8D11A11
:105060008269914206D2011D286907E09A4203D263
:10507000994201D3012403E0011DE86800F063FABE
:10508000204670BD5C00002010B5044600F080FA98
:10509000A06B28B15FF0000400F09AFA204610BD22
:1050A0000124F9E730B589B03C4D6EE00498002842
:1050B00006DADDE90601059A90470498002864DBCA
:1050C000069C606910B1201D00F004FA03A800F0EE
:1050D000D7F8024604980A2857D2DFE800F0050501
:1050E000052D334A05052D3394F8280040F00100C2
:1050F00084F828000599A069059B01442046FFF724
:10510000A7FF68B3216A2046884794F82800400723
:105110003BD5002000900598A1690023421819464C
:10512000204601F0D1FAD8B9502080F31188BFF39E
:105130004F8FBFF36F8FFEE714F8280F20F00100A8
:10514000207022E094F8280040F0010084F8280044
:105150000598A06128B1811813462046FFF778FF13
:1051600013E0502080F31188BFF34F8FBFF36F8F90
:10517000FEE794F82800810703D4204600F03CFAAB
:1051800003E020F0010084F82800002204A9286828
:1051900000F0A4FE002889D109B030BD5C000020D9
:1051A0002DE9FC410F46054600F006FC01A800F081
:1051B00067F80446019818B101F0F4F9BDE8FC81E4
:1051C000254EAFB130690068D0B30027291B3A469D
:1051D000306800F093FA01F0E5F90028EED11F499C
:1051E0004FF080500860BFF34F8FBFF36F8FE5E73C
:1051F000A542EBD801F0D6F9F0682746C068C4682C
:10520000201D00F067F994F82800410719D5A0691E
:105210002B4641193A462046FFF71AFFA8B1002055
:105220000346014600902A46204601F04DFA60B937
:10523000502080F31188BFF34F8FBFF36F8FFEE7CD
:1052400007E020F0010084F82800216A2046884702
:10525000B4E70127BAE700005C00002004ED00E09D
:105260000648C16B096829B1C16BC968C96849683A
:10527000816270474FF0FF31FAE70000180000200C
:1052800070B5054601F05EF8064E0446B0688442EB
:1052900003D200F009F8012000E000202860204639
:1052A000B46070BD5C000020F8B5194D20E0C06806
:1052B000C4680668201D00F00DF9216A2046884761
:1052C00094F82800400713D5A0693044B04206D9AD
:1052D00024616060211DE86800F035F908E00020D5
:1052E0000346014600903246204601F0EDF938B100
:1052F000E86801680029DAD12969C5E90310F8BD19
:10530000502080F31188BFF34F8FBFF36F8FFEE7FC
:105310005C00002008484068401C4FF0500080F3BB
:10532000118804D0BFF34F8FBFF36F8FFEE7BFF339
:105330004F8FBFF36F8FFEE794000020074CE068AB
:10534000016841B1C0680021D0F80000FFF728FFD4
:10535000FFF7A8FEF3E701210020F7E75C0000203B
:105360002DE9F041044600F013F994F9455004F199
:10537000240609E0606A48B1304601F0DBF808B164
:1053800000F09AFA6D1E6DB2002DF3DC4FF0FF367F
:1053900084F8456000F01CF900F0FAF894F94450E4
:1053A00004F1100709E0206948B1384601F0C2F85D
:1053B00008B100F081FA6D1E6DB2002DF3DC84F8A7
:1053C0004460BDE8F04100F003B900002DE9F04170
:1053D0000546002700F0F0FA324E306808B9FFF7B2
:1053E00051FD706905424ED1C5B3083568070ED02E
:1053F00005F00700C0F108000544680707D05020F9
:1054000080F31188BFF34F8FBFF36F8FFEE72DB38B
:105410007068854237D82348183001460C6801E08F
:1054200020460C466168A94202D221680029F7D1C2
:1054300031688C4227D007682168016060680837AE
:10544000411B10290FD96019420708D0502080F362
:105450001188BFF34F8FBFF36F8FFEE713E04160FA
:105460006560FFF7CFFD61687068401A7060B268D0
:10547000904200D2B060706901430020C4E900018D
:10548000F068401CF06001F08DF8780707D05020DC
:1054900080F31188BFF34F8FBFF36F8FFEE738465D
:1054A000BDE8F0817400002010B5031F4FF0807438
:1054B0001C601B1F21F001011960191F044B0B60B8
:1054C00014390A60091F6FF0020244380A6010BDE7
:1054D00015530008D0E9013201699A60D0E901232F
:1054E0005A604A68824201D182684A6000220261A1
:1054F0000868401E0860086870470000034B03609E
:1055000003F164000860802010607047EC0D0020FB
:10551000044B036003F1640008604FF48070106076
:105520007047000050100020704700F108014FF054
:10553000FF32C0E90112C1600161002101607047C2
:1055400000210161704730B50B685A1C02D000F190
:10555000080202E0026904E02246546825689D4280
:10556000FAD953684B6099608A605160086101689C
:10557000491C016030BD42684A6093688B60936843
:105580005960916008610168491C01607047000022
:10559000502080F31188BFF34F8FBFF36F8F0A49FC
:1055A0004868401C486001280CD10848006810F089
:1055B000FF0F07D0502080F31188BFF34F8FBFF348
:1055C0006F8FFEE7704700009400002004ED00E0BC
:1055D0000849486828B1401E486001D180F311880D
:1055E0007047502080F31188BFF34F8FBFF36F8F48
:1055F000FEE700009400002070B500282AD0164D68
:10560000A0F1080460686969084207D1502080F35E
:105610001188BFF34F8FBFF36F8FFEE722683AB157
:10562000502080F31188BFF34F8FBFF36F8FFEE7D9
:105630008843606000F0C0F9606869680844686089
:105640002046FFF7DFFC2869401C2861BDE8704058
:1056500000F0A8BF70BD0000740000204FF0E020F3
:1056600000210161816105494FF47A720968B1FB3B
:10567000F2F1491E416107210161704714000020C9
:1056800010B5FAF72FFE114910280ED300F1E020D3
:1056900090F8F0030A78904207D2502080F31188E6
:1056A000BFF34F8FBFF36F8FFEE70948006889682B
:1056B00000F4E060884207D9502080F31188BFF3DE
:1056C0004F8FBFF36F8FFEE710BD000094000020E6
:1056D0000CED00E010B5084B002200BF53F832403B
:1056E0001CB1521C082AF9D310BD43F8321003EB49
:1056F000C201486010BD0000D007002070B51546FB
:105700000E460446FFF744FF94F944100020491C5C
:1057100001D184F8440094F94510491C01D184F862
:105720004500FFF755FFA06B28B92A46314604F122
:10573000240000F0DFF82046BDE87040FFF710BEFF
:1057400010B5020014D00F48006B38B1502080F320
:105750001188BFF34F8FBFF36F8FFEE700F02CF976
:1057600000211046FFF768FA00F01CFF002807D15F
:1057700005494FF080500860BFF34F8FBFF36F8F24
:1057800010BD00001800002004ED00E070B50D46CB
:1057900004000BD095B11E4A106BB8B1502080F3B5
:1057A0001188BFF34F8FBFF36F8FFEE7502080F358
:1057B0001188BFF34F8FBFF36F8FFEE7502080F348
:1057C0001188BFF34F8FBFF36F8FFEE700F0F4F83F
:1057D000D26823685919934204D98B420AD991425D
:1057E00002D807E08B42FAD9881A21600021FFF71E
:1057F00023FA00E0216000F0D5FE002807D105491A
:105800004FF080500860BFF34F8FBFF36F8F70BDB4
:105810001800002004ED00E070B50546FFF7B8FE63
:105820001E4C05B92568281DFFF754FEA86A18B15B
:1058300005F11800FFF74EFE606A401C60622068A8
:10584000854207D1291D1648FFF795FE6068401C68
:10585000606007E0A068401EA0602846FFF7F7FAE6
:10586000FFF7FEFCFFF7B4FE6069002814D0206843
:10587000854211D1206B38B1502080F31188BFF3DD
:105880004F8FBFF36F8FFEE706494FF080500860DF
:10589000BFF34F8FBFF36F8F70BD00001800002063
:1058A000AC0C002004ED00E002490A6A0260C968FD
:1058B000416070471800002001490120C86170470D
:1058C0001800002010B50C4650B10949096818317C
:1058D000FFF739FE2046BDE810400121FFF7ACB9C3
:1058E000502080F31188BFF34F8FBFF36F8FFEE717
:1058F0001800002070B514460D4668B10A490968C1
:105900001831FFF738FE0CB14FF0FF35214628461D
:10591000BDE87040FFF790B9502080F31188BFF3C5
:105920004F8FBFF36F8FFEE71800002030B587B0B0
:105930000024039405AA04A903A80494FFF7DEFD3C
:10594000DDE903010094CDE90110002316A11848F8
:10595000059A00F0C6FB174D0028E86221D000F040
:1059600083FE012809D0401C1BD1502080F31188F0
:10597000BFF34F8FBFF36F8FFEE7502080F3118886
:10598000BFF34F8FBFF36F8F4FF0FF30A86201203E
:105990006861EC60FEF73CFF07B0BDE8304000F006
:1059A00065B807B030BD000049444C450000000018
:1059B000D14E0008180000200248016B491C016309
:1059C000704700001800002010B5264C206B10B165
:1059D0000120E06110BD0020E061FEF755FFA063EB
:1059E000626B904204D92168821A8B6D1A448A65D1
:1059F000606320684FF0A531006B02688A4208D1CD
:105A000042688A4205D182688A4202D1C0688842CF
:105A100004D0216820683431FFF786FD20691249DF
:105A200001E0B8B1401E00EB800251F82220002AAC
:105A3000F7D000EB800201EB820101F108034A6814
:105A400052684A609A4201D152684A60D168216026
:105A5000206110BD502080F31188BFF34F8FBFF33A
:105A60006F8FFEE718000020100800201CB5374893
:105A70000168374A914207D1502080F31188BFF363
:105A80004F8FBFF36F8FFEE700683149491E884290
:105A900007D1502080F31188BFF34F8FBFF36F8F72
:105AA000FEE72C4908780190FF20087008788DF8EF
:105AB00000009DF800009DF8002000F0F0009042EA
:105AC00007D0502080F31188BFF34F8FBFF36F8F43
:105AD000FEE79DF80000204C00F0500020700720E9
:105AE000A06005E09DF8002052008DF80020401EC7
:105AF0009DF800201206F5D4A060032807D050209E
:105B000080F31188BFF34F8FBFF36F8FFEE74FF421
:105B10004070A060019808700C482030016841F482
:105B200070010160016841F070410160FFF796FD6E
:105B300000206060FAF79EFB0848016841F0404190
:105B40000160FAF783FB00201CBD000000ED00E0BF
:105B500071C20F4100E400E09400002034EF00E047
:105B600010B5502080F31188BFF34F8FBFF36F8FB4
:105B700000F0F6FB18B104494FF080500860002097
:105B800080F3118810BD000004ED00E0F8B5174661
:105B90000E46050013D005FB06F05030FFF716FC4B
:105BA00004000AD0002084F8460004F150023B466D
:105BB000314628460094FFF7BBF92046F8BD502037
:105BC00080F31188BFF34F8FBFF36F8FFEE738B5B7
:105BD000049D18B153B1CAB181B120E0502080F3C7
:105BE0001188BFF34F8FBFF36F8FFEE7502080F314
:105BF0001188BFF34F8FBFF36F8FFEE7502080F304
:105C00001188BFF34F8FBFF36F8FFEE739B150207C
:105C100080F31188BFF34F8FBFF36F8FFEE75024DF
:105C20001C46012384F846302B460094FFF780F988
:105C3000204638BD70B50D46040025D0FFF7A8FCFE
:105C4000D4E90F20216802FB0011A1600021A163AB
:105C5000216861600A46D4E90F01401E00FB012162
:105C6000E16021464FF0FF3001F8440F487004F125
:105C700010008DB1FFF759FC04F12400FFF755FC2B
:105C8000FFF7A6FC012070BD502080F31188BFF300
:105C90004F8FBFF36F8FFEE721690029F0D000F02E
:105CA00049FC0028ECD004494FF080500860BFF355
:105CB0004F8FBFF36F8FE3E704ED00E02DE9FF475F
:105CC00082B01D468A464FF00008040003D0BAF1A6
:105CD000000F08D011E0502080F31188BFF34F8FE0
:105CE000BFF36F8FFEE7206C38B1502080F311882E
:105CF000BFF34F8FBFF36F8FFEE7022D0AD1E06B2A
:105D0000012807D0502080F31188BFF34F8FBFF3D5
:105D10006F8FFEE700F008FB3F4F4FF000094FF098
:105D2000805648B9049838B1502080F31188BFF3E9
:105D30004F8FBFF36F8FFEE7FFF72AFCA06BE16B7D
:105D4000884207D3022D05D00498D0B1B8F1000FD6
:105D50001AD01EE02A4651462046FFF742F8616AF3
:105D600019B104F1240000F0E5FB20B13E60BFF35F
:105D70004F8FBFF36F8FFFF72BFC012006B0BDE8FC
:105D8000F087FFF725FC22E06846FFF78DFD4FF016
:105D90000108FFF71DFCFFF70FFEFFF7F9FB94F971
:105DA0004400401C01D184F8449094F94500401C03
:105DB00001D184F84590FFF70BFC04A9684600F078
:105DC00029F930B12046FFF7CBFA00F0EBFB0020B9
:105DD000D4E7FFF7DDFBA06BE16B884213D1FFF73F
:105DE000F7FB04F110000499FFF76CFD2046FFF764
:105DF000B7FA00F0D7FB00289ED13E60BFF34F8F6B
:105E0000BFF36F8F98E7FFF7E3FB2046FFF7A8FA91
:105E100000F0C8FB90E7000004ED00E02DE9F0473A
:105E20001F4690468946040003D0B9F1000F08D000
:105E300011E0502080F31188BFF34F8FBFF36F8FB5
:105E4000FEE7206C38B1502080F31188BFF34F8FEC
:105E5000BFF36F8FFEE7022F0AD1E06B012807D056
:105E6000502080F31188BFF34F8FBFF36F8FFEE791
:105E7000FFF706FC5020EFF3118680F31188BFF383
:105E80004F8FBFF36F8FA06BE16B884206D3022F59
:105E900004D0002086F31188BDE8F08794F94550BE
:105EA000A06B3A4649462046FEF79BFF681C04D08B
:105EB0006D1C84F845500120ECE7606A0028FAD098
:105EC00004F1240000F036FB0028F4D0B8F1000FF4
:105ED000F1D00121C8F80010EDE700002DE9F747E7
:105EE000002683B08A46040003D0BAF1000F08D020
:105EF00011E0502080F31188BFF34F8FBFF36F8FF5
:105F0000FEE7206C38B1502080F31188BFF34F8F2B
:105F1000BFF36F8FFEE700F007FADFF8F4804FF071
:105F200000094FF0805748B9059838B1502080F3E8
:105F30001188BFF34F8FBFF36F8FFEE7FFF728FB8A
:105F4000A56BC5B151462046FEF738FF6D1EA5630F
:105F5000206950B104F1100000F0ECFA28B1C8F843
:105F60000070BFF34F8FBFF36F8FFFF731FB01203E
:105F700006B0BDE8F087059808B11EB106E0FFF74E
:105F800027FB27E06846FFF78FFC0126FFF720FB81
:105F9000FFF712FDFFF7FCFA94F94400401C01D111
:105FA00084F8449094F94500401C01D184F8459050
:105FB000FFF70EFB05A9684600F02CF800282046E4
:105FC0000AD0FFF7CDF900F0EDFA2046FFF75CF8B4
:105FD0000028B3D00020CBE7FFF756F890B104F1CA
:105FE00024000599FFF76EFC2046FFF7B9F900F091
:105FF000D9FA0028A2D1C8F80070BFF34F8FBFF3C1
:106000006F8F9BE72046FFF7ABF900F0CBFA95E7DF
:1060100004ED00E02DE9F0410C46050011D0C4B1BB
:10602000FFF7B6FA174BDA686E682068911B471CB9
:1060300017D02F681B6A9F4219D0964217D80124A7
:1060400010E0502080F31188BFF34F8FBFF36F8FA4
:10605000FEE7502080F31188BFF34F8FBFF36F8F9F
:10606000FEE70024FFF7B4FA2046BDE8F08188423D
:1060700005D9401A20602846FFF716FCF1E70020FA
:106080002060DCE7180000202DE9FF5F8346DDE992
:106090000E87994616468A469000FFF797F9050045
:1060A0001CD06420FFF792F9040014D0002025636F
:1060B00084F86100CDE90240CDE900874B463246C5
:1060C00051465846FEF745FF2046FEF7E3FD012006
:1060D00004B0BDE8F09F2846FFF78EFA4FF0FF307E
:1060E000F6E7F0B585B0DDE90B640A9DA6B1DCB139
:1060F000642700972663022684F86160002604AFB7
:10610000CDE90246CDE90057FEF723FF2046FEF712
:10611000C1FD049805B0F0BD502080F31188BFF395
:106120004F8FBFF36F8FFEE7502080F31188BFF3CE
:106130004F8FBFF36F8FFEE72DE9F0411F4690466A
:106140000D46012690B10446FFF722FA0FB1E06D2B
:10615000386094F86000022184F86010B8F1050FEF
:1061600019D2DFE808F0230B0E141200502080F340
:106170001188BFF34F8FBFF36F8FFEE7E16D2943A7
:1061800001E0E16D491CE16510E0022801D0E56500
:106190000CE0002634E0E16D491C07D0502080F36C
:1061A0001188BFF34F8FBFF36F8FFEE7012827D110
:1061B000201DFFF78FF9154DE06A2969884200D943
:1061C0002861134900EB800001EB8000211DFFF7DF
:1061D000D2F9A06A38B1502080F31188BFF34F8FF5
:1061E000BFF36F8FFEE7E06A2968C96A884207D962
:1061F00008494FF080500860BFF34F8FBFF36F8F97
:10620000FFF7E6F93046BDE8F081000018000020F5
:106210001008002004ED00E02DE9F0471F46DDF8EE
:10622000209092460D4604004FF001081AD0FFF767
:1062300027FA5020EFF3118680F31188BFF34F8FB8
:10624000BFF36F8F0FB1E06D386094F860000221EA
:1062500084F86010BAF1050F1AD2DFE80AF0240BB7
:106260000E141200502080F31188BFF34F8FBFF33C
:106270006F8FFEE7E16D294301E0E16D491CE165A7
:1062800011E0022801D0E5650DE04FF0000839E08B
:10629000E16D491C07D0502080F31188BFF34F8F68
:1062A000BFF36F8FFEE701282CD1A06A38B15020D0
:1062B00080F31188BFF34F8FBFF36F8FFEE7144D4C
:1062C000286B18B104F1180112480DE0201DFFF7EA
:1062D00001F9E06A2969884200D928610E4900EB7A
:1062E000800001EB8000211DFFF745F9E06A296875
:1062F000C96A884206D90120B9F1000F01D0C9F856
:106300000000E86186F311884046BDE8F087000090
:1063100018000020980C0020100800200148006898
:1063200070470000180000200548416919B1006B52
:1063300018B100207047012070470220704700000C
:10634000180000200148C0687047000018000020B5
:1063500010B5FFF795F90148C06810BD180000207E
:106360002DE9F0412E4C0027206B28B1A069401C7C
:10637000A0613846BDE8F081E668761CE66013D17E
:10638000E06B006838B1502080F31188BFF34F8F65
:10639000BFF36F8FFEE7E06B216CE1632064206A3E
:1063A000401C2062FEF75CFFA06ADFF8788086421E
:1063B00009D3E06B0068A0B1E06BC068C56868688D
:1063C000864211D2A0622068C06A00EB800158F8B2
:1063D0002100012800D90127E0690028C9D0012740
:1063E000C7E74FF0FF30EDE7281DFFF773F8A86A05
:1063F00018B105F11800FFF76DF8E86A21698842C5
:1064000000D9206100EB800108EB8100291DFFF716
:10641000B2F8E86A2168C96A8842CAD30127C8E786
:1064200018000020100800202DE9F0411E461546F6
:1064300088460746FFF7ACF81C4C206890F86000CF
:10644000022814D02068C16DB943C16521680120BC
:1064500081F860005EB101213046FEF7EDFB144982
:106460004FF080500860BFF34F8FBFF36F8FFFF77F
:10647000AFF8FFF78DF815B12068C06D286020686F
:1064800090F86000022801D0002505E02068C16D69
:1064900021EA0801C16501252168002081F860001A
:1064A000FFF796F82846BDE8F081000018000020AC
:1064B00004ED00E070B504004FF0000133D01B4D37
:1064C0002868844207D0502080F31188BFF34F8F93
:1064D000BFF36F8FFEE7606D38B1401E6065236DBE
:1064E000E26A9A421FD040B11DE0502080F311882B
:1064F000BFF34F8FBFF36F8FFEE7201DFEF7EAFF5C
:10650000206DE062C0F13800A061E06A296988422C
:1065100000D92861064900EB800001EB8000211DB5
:10652000FFF729F80121084670BD0000180000207F
:106530001008002070B5C068C46854B104F1180098
:106540000646FEF7C7FF144D286B50B1314613487D
:1065500015E0502080F31188BFF34F8FBFF36F8F8A
:10656000FEE7201DFEF7B6FFE06A2969884200D9E0
:1065700028610B4900EB800001EB8000211DFEF734
:10658000FAFFE06A2968C96A884202D90120E861F5
:1065900070BD002070BD000018000020980C002085
:1065A000100800202DE9F0472C4D00242746286BC9
:1065B00038B1FEF7EDFF286B401E2863286B40B111
:1065C00046E0502080F31188BFF34F8FBFF36F8FE9
:1065D000FEE7A968224E0120D1B3A6F59169804655
:1065E0003068E0B1F068C46804F11800FEF772FF8B
:1065F000201DFEF76FFFE06A2969884200D92861F3
:1066000000EB800109EB8100211DFEF7B4FFE06A79
:106610002968C96A8842E3D3C5F81C80E0E70CB159
:10662000FEF71EFEAC694CB14FEA0806FFF798FE74
:1066300000B1EE61641EF9D10020A861E86938B1AB
:106640000849012738070860BFF34F8FBFF36F8FEA
:10665000FEF7BEFF3846BDE8F087000018000020B6
:10666000980C002004ED00E010B586B0FEF77AFB30
:10667000114C2068B8B100200390049005AA04A929
:1066800003A8FEF745FFDDE9032102208DE807009E
:1066900000230AA10B48059AFFF723FD606010B1A3
:1066A00006B0012010BD502080F31188BFF34F8F3A
:1066B000BFF36F8FFEE700005C000020546D722076
:1066C000537663003D5300082DE9FF411E461346F3
:1066D00002000A9D4FF0000016D0144C2768002FCE
:1066E0000FD0CDE900130292062917DAFFF71CFE3E
:1066F00002284FF000030FD0002269462068FFF700
:10670000DDFA04B0BDE8F081502080F31188BFF3BA
:106710004F8FBFF36F8FFEE72A46EEE70023324626
:1067200069463846FFF77AFBEBE700005C00002083
:1067300021F00042A2F16052B2F5801F01F0004347
:1067400028BFD2F17F6C0BD95FEA001C43EAC2027A
:1067500042EB507018BF704728BF20F0010070470F
:10676000B2F5801FBCBF184670474FEA410C1CF5BC
:10677000001F02D2084600F04FBB70B500F04CFA83
:1067800000000089FFF7F6BF4FF00040A0F5800041
:10679000704700002DE9C04130B4DFF8A0C23CEAE8
:1067A000111418BF3CEA131400F0EC8081EA0305D1
:1067B0001CEA111444EAD57418BF1CEA131500F042
:1067C000C780A4EB05044FF0004545EAC12145EA26
:1067D000C32341EA505143EA525304F17F74994272
:1067E00004F500344FEAC0204FEAC22208BF9042AD
:1067F00000F09C804FEA13650FF24016765D4FEA79
:10680000134506FB05F7C7F1807706FB07F74FEA4C
:10681000D737A7FB03687642C8F58038A7FB06CEBA
:1068200038BFA8F1010807FB08E64FF0000EA6FBF1
:10683000028CE6FB03CEDCF1000CCEF1004E38BF3B
:10684000AEF1010EA6FB0C584FF000074FF000050B
:10685000E6FB0E87A1FB08C6A0FB07CE16EB0E06D3
:1068600045F10005E1FB076515F1E04E7EBFA4F59B
:1068700080345FEA46066D4116F1800745F1000558
:106880004FEA17274FEA066647EA0567A6F1DE4694
:10689000B6F1805F4FEA15251FD9384624F0010C68
:1068A00005EBC471BCF1FE6F01EB0C1102D8F0BC1A
:1068B000BDE8008124425CBF01F5801E9EEAC47FD2
:1068C00002D4F0BCBDE80081244238D4F0BCA1F170
:1068D000C041BDE8004100F0EDB94FEAD22242EAE2
:1068E00043524FEAD323A7FB02864FEAD02040EA67
:1068F000415007FB03661EEA0E0F4FEAD12105FB4C
:10690000026658BFA6EB0056B6EB00564FEA520E91
:106910004EEAC37E18EB0E0E56EB530EBDD518EBA8
:1069200002085E417F1C55F10005B6E74FF4801563
:106930004FF000074FF000064FF00008ADE7F0BC45
:106940004FF0000001F1C04101F00041BDE80081BD
:1069500011EA0C1F0CEA131500D00CE013EA0C1F0F
:1069600000F025804FF00000F0BC81EA030101F047
:106970000041BDE80081F0BCBDE8004181EA0301AF
:1069800000F098B9F0BCBDE8004170B500F044F9E2
:10699000097EFC3E00F007B881EA03014FF00000D9
:1069A00001F00041704781EA030100F083B9F0BCB7
:1069B000BDE800414FF0000021497047FFFDFBF9A1
:1069C000F7F5F4F2F0EEEDEBE9E8E6E4E3E1E0DE22
:1069D000DDDBDAD8D7D5D4D3D1D0CFCDCCCBCAC894
:1069E000C7C6C5C4C2C1C0BFBEBDBCBBBAB9B8B7BB
:1069F000B6B5B4B3B2B1B0AFAEADACABAAA9A8A8AE
:106A0000A7A6A5A4A3A3A2A1A09F9F9E9D9C9C9B7B
:106A10009A99999897979695959493939291919026
:106A20008F8F8E8E8D8C8C8B8B8A898988888787B7
:106A30008685858484838382828181800000FF072C
:106A40000000F87F4FEA1153A3F58063D3F11E03D2
:106A5000A8BFD3F1200C08DB4FF0004242EAC1226C
:106A600052EA505232FA03F0704709420BD4102B0D
:106A7000C4BF0020704703F5787CBCF1FF3F05D010
:106A80004FF0FF3070474FF00000704770B500F0D6
:106A9000C3F800BF4992248000207047F0E7B0FAA5
:106AA00080F310FA03F10AD0C3F11D0303F58063EC
:106AB0004FEA41504FEA035202EBD12170474FF0A9
:106AC00000007047DFF848C170B51CEA111E1EBFF8
:106AD0001CEA13159EEA0C0F95EA0C0F00F06F806C
:106AE00081EA030423EA4C134EEAD47E21EA4C11D6
:106AF00041F4801143F48013AE44A1FB024CA0FB8F
:106B00000365AEF17F7E361955EB0C05A1FB034CF6
:106B10004CF10003A0FB021C16EB0C06654153F17F
:106B20000003094218BF46F0010613F4007F0BD1A1
:106B30004FEA03314FEA0530340341EA155140EA88
:106B400016506FF003020AE04FEAC3214FEAC52056
:106B5000F40241EA555140EA56506FF0020202EB4E
:106B60002E4201EB025585EACE710AD05FEA440C51
:106B700018BF24F0004450F1000041F1000120EA68
:106B8000D47040F2FE7C624500D270BDA84214BFB2
:106B90004FF080444FF04044002E08BF0024BEF167
:106BA000806FA8BFA1F1C041BDE8704080F2828033
:106BB0004FF0000001F1C04101F0004170479EEA32
:106BC0000C0F0CEA131518BF95EA0C0F06D04FF006
:106BD000000081EA030E0EF0004170BD00F01CF8C9
:106BE0008900013E00F007B800F009B84FEA430CF5
:106BF0005FEA5C5C08D081EA030100F05BB84FEA11
:106C0000410C5FEA5C5CF6D14FF00000014970472F
:106C10000000FF070000F87F0EF1020E2EF0030EB9
:106C20005EF8046B364205D4012A43EB030515F5E3
:106C3000001F12D8012841EB010C1CF5001F0CD8D5
:106C40000ED14FEAD17C15F5001F0CEB4C0C0CF16A
:106C5000020C08BF4CEBD37C04E04FF0080C01E0C1
:106C60004FEAD37C0CEB4C0526FA05F606F0070636
:106C7000B6F1040C06D20EEB860CBDE870404CF069
:106C8000010C6047DFE80CF0090B02024FF00041F5
:106C90004FF00000A1F5002170BD194610460128F3
:106CA00051EB010418BFD4F5001484BF002001F09B
:106CB000004170BD0808A0F500114FEA310170478E
:106CC00043004FEAD30C4FEA3C0C43401FBF400740
:106CD0000CF1605113F0FE4F70471CF0006F03D1B0
:106CE00000200CF0004170470CF0004343EA507064
:106CF00010B540EACC0000F044F800BF000000925C
:106D00004FEA0001FFF7D6BF4FF000414FF00000FF
:106D1000A1F500217047000000EE100A00EE901A65
:106D2000B4EE600AF1EE10FA78BF704700F00DB8CB
:106D300010B5FFF7F1FFEFF3008020F0104038BFEF
:106D400040F0004080F3008810BDBDE8104010B551
:106D500000F017F80000000900F007B84FF04040BD
:106D600010F1004FEFF300807047401058BFC0F1A2
:106D70004040491058BFC1F140418142EFF30080CB
:106D800070470EF1020E2EF0030E5EF8044B244203
:106D900004D44FEA4102B2F17F4F11D84FEA4003C9
:106DA000B3F17F4F0CD80ED14FEAD07CB2F17F4FB8
:106DB0000CEB4C0C0CF1020C08BF4CEBD17C04E04A
:106DC0004FF0080C01E04FEAD17C0CEB4C0324FAA5
:106DD00003F404F00704B4F1040C06D20EEB840CA7
:106DE000BDE810404CF0010C6047DFE80CF00708EC
:106DF00002024FF00040A0F5800010BD084642009E
:106E000018BFD2F1807288BF00F0004010BD4FF073
:106E10004070E1EE100A7047FF2141EAD050C005F2
:106E200070470000D06E0008000000000000000065
:106E30000000000000000000000200001800000038
:106E400000000000000000000006101600061016EA
:106E5000000000000000000001020304060708090A
:106E60000000000001020304DC6E000800000000C6
:106E7000000000000000000000000000000400000E
:106E8000300000000000000000000000E86E000874
:106E900000000000000000000000000000000000F2
:106EA00000040000180000000000000000000000C6
:106EB000000000006E83F9A22915444ED15727FC2B
:106EC000C0DD34F5999562DB4190433CAB6351FEE4
:106ED00064656661756C745461736B005461736BA7
:106EE0005F496E6974000000636861737369735F62
:106EF000636F6E74726F6C00186F000800000020E2
:106F0000B0000000C4010008C86F0008B0000020F5
:106F100008800000E0010008000000000000000000
:106F20000100000010000000000000000024F40038
:106F30000000000000000000000000000000000051
:106F40000000000000000000000000000000000041
:106F50000000000000000000000000000000000031
:106F60000000000000000000000000000000000021
:106F70000000000000000000000000000000000011
:106F80000000000000000000000000000000000001
:106F900000000000000000000000000000000000F1
:106FA00000000000000000000000000000000000E1
:106FB000AAAAAAAA00000000000000000000000029
:086FC0000000000000000000C9
:040000050800018965
:00000001FF
